:020000041100E9
:10300000002373B52B4D2C4C28006361022601F080
:1030100065F94021FE2221742800284B009601F01A
:10302000AFF9002836D1217CFF222800244B0096DE
:1030300001F0A6F900282DD1224BA2899A4226D16F
:10304000E389214A93420DD1204B6361204B2268D2
:10305000002A03D1002B01D043CB43C4280001F048
:103060007BF973BD1B4A934201D00023EFE71A4B53
:103070001A4A1B68934206D9C02304222800217CE7
:103080009B0001F0F3F9114B6361154BDFE700235F
:103090002374EAE7CC233821AC2228009B01217459
:1030A00001F0E4F90028F2D10E4B63610E4BE3818D
:1030B0000E4BCCE7643CFF1F085CFF1F145CFF1F36
:1030C000165CFF1F595900008305000009410011DB
:1030D0009CBC0011821500002C5CFF1F87130000B0
:1030E000A8BC0011C1410011AAAAFFFF90BC0011A9
:1030F000F7B5164B0192C318021D002000938823D8
:103100005B05D3181B685C1C1AD09CB2402C18D8E5
:103110008D781E0CAC466746CD782D023D43AE42FD
:1031200006D1019800280ED110000C70240A4C70B2
:1031300003249BB20733A343D218009B9A42DED3E9
:10314000FEBD4432F9E71000FAE7C046FC0F00006C
:10315000802213B503000324019189B25201073183
:103160009B18A14304305A1A88235B05C3181B68B7
:10317000591C03D190429241104016BD99B240298A
:1031800007D80B000733A343C0189042ECD30020AC
:10319000F3E74430F9E7134B134A1B68126810B584
:1031A000FA24934201D81A00F824104BE4021B6859
:1031B0009A4210D813000E4A12689A420ED3013375
:1031C00007D1F823DB029C4203D10A49054808F0E5
:1031D00083FA200010BDFC24E402ECE7FE24E402A4
:1031E000F7E7C04600C0071100D0071100E0071143
:1031F00000F00711FFFFFF7FF0B59BB015000490B2
:103200000391402A00D9A0E006AB59801A80FFF74D
:10321000C2FF0400042816D9002206A9FFF768FFA0
:10322000052810D906AB1B88AB420CD1002D07D066
:10323000514B2A000499C01808F0FEFA002802D168
:1032400001201BB0F0BD06AB1D8020000699FFF7E2
:103250007FFF041E7BD1069B0793FFF79CFF802313
:103260005B01C618802307001B039E4201D3F8268A
:10327000F60288235B05F31801931B68013302D023
:10328000019808F079FB3D49019808F025FA3B1DAB
:103290000293331D05938822029B52059B181B68DD
:1032A00008935A1C3CD044219AB20091402A04D879
:1032B0000320D11D814389B2009103991B0C8B42DD
:1032C00024D0402A22D80122300008A9FFF710FF9D
:1032D000021E1BD1380008A9FFF70AFF04000428CA
:1032E00031D9009A059B9B1880225201B218934253
:1032F00040D288235B05C118009A09A808F0E4FBB6
:103300001D4B009A09A9F01808F00EFC009A029BC8
:103310009446634402931A4B029AFB189A42BAD31A
:1033200088235B05FC1821680198013908F0D4F95D
:10333000200008F021FB039A07AB5A803000079960
:10334000FFF706FF0400002C03D1002079E70428D2
:10335000FBD988235B05E018069908F0BDF9032323
:10336000EA1C9A4300D16BE7034B0499E01808F07C
:10337000DBFB65E70424ECE704000011FFFFFF7F9F
:10338000F80F0000F7B505001400402A21D80027E7
:1033900001AE71803780FFF7FEFE042816D93A008F
:1033A0003100FFF7A5FE042810D93688BC420BD0A7
:1033B000BD4209D0221CB44200D9321C064B92B245
:1033C000C118280008F080FB30B2FEBDC04300B237
:1033D000FBE703204042F8E70400001137B5042260
:1033E00004000D0001A81649FFF7CCFF02000428D5
:1033F0000BD1019BA34208D3AB4204D0104901A8D2
:103400000195FFF7F9FE01203EBD0E4C2368200018
:10341000019308F0B1FA019920000139019108F0F7
:103420005BF980235B01E418074B9C42EED1042238
:10343000034901A80195FFF7DFFE0020E4E7C0463D
:103440005555000000C007110000081130B589B0C3
:1034500008F092F810226946254808F0CDF9254B6E
:10346000009A9A420ED1019B029A0F2B33D8002169
:1034700001240698013B08D2002900D00292029B49
:10348000013331D10023029325E0551CF2D1020013
:103490002100EFE710341022200004A908F0ACF955
:1034A000029B013301D1069B0293882304995B059B
:1034B000C918059B06981A03120B049105928142C4
:1034C00003D02B4201D108F0FFFA019B013B01938D
:1034D000019B002BDED1029B002B03D004930498A8
:1034E0004168084709B030BDE025014C2D03EFE7E6
:1034F00000000111504859368022F8B5964C974B80
:10350000D200002120001C6008F036FB2300944A02
:1035100088331A60934B1A786A23002A00D011333B
:10352000E3620A232365904B37221B780821A363AB
:103530008E4B6018E361102323628D4B3B25636142
:10354000C823DB00A36123008C331A602823013ACF
:10355000E26321646364C267043A201DC2672000ED
:10356000BC3005602000C03001602000C430036022
:1035700020000635CC3005602000083DC8300560CD
:103580002000D03002602200D43211602200D832F4
:10359000136022000226E032200016604222DC3056
:1035A000026020001B3DE43005602000E83001602F
:1035B0002000EC30036023000520F4331860230062
:1035C000F0331A602300183290331A6023009433CA
:1035D000196023001E3A98331A60AF23DB00236082
:1035E000644BFA252363644B6448A3642300B93217
:1035F000FC33FF32AD00A260E56022611D60A06275
:103600007320E0656D386065A065FA2796203F015C
:103610008000E76465625960A0660920E0660020CA
:10362000616757496666E167564E57492667A06746
:103630000F601527676027001A219C373960270023
:103640000731A037396027004B49A837396021007E
:10365000F8310D6021006427A4310F6021005F3F25
:10366000AC310F602100033FB0310F602700B43749
:103670003D00C8272F6027003825B83738609D6087
:10368000424D96215D64424D8900DD61414D1962D4
:103690005D62F53DFF3D9D621E253949DD66596637
:1036A000996499673C49DE651E6618675867D96753
:1036B000BE233A495B00E1508130394BFF30235043
:1036C00004302150C42149006350C623E4205B002C
:1036D000E2500433E2503349334A344BD160344929
:1036E000800019503349E938FF3819503249043005
:1036F000195032493248D16132491163324951631C
:103700001900F4310860CE20304940001160304982
:10371000195019002F48F83108602F49D1658221CE
:103720002E4A89005A501A002D490832D1671A00D2
:103730002C49B432116088212B4A89005A501A0052
:103740002A49883211602A4ADA6408F0EDF801202B
:1037500008F09AF8F8BDC0460004FF1FAC5EFF1FDA
:103760009069FF1F9C3EFF1F4A0AFF1F3A07000097
:1037700080C3C9019A02000050C300006A1800000B
:1037800088130000204E0000F009FF1F6509FF1F8D
:1037900068100000C4090000DC05000040420F0072
:1037A00010270000D91AFF1FFC00FF1F0000FF1F99
:1037B0008127FF1FC52AFF1F5D29FF1F251EFF1F31
:1037C0007523FF1F411EFF1FED1FFF1FB11DFF1FB0
:1037D0000124FF1FE924FF1FD918FF1FB923FF1F72
:1037E000C921FF1FD521FF1FB11CFF1F691DFF1F2E
:1037F0009D1CFF1F0223F0B501245C4D5C4E2B7015
:103800005C4B91B01C705C4F039333680021200027
:10381000FB7006F0D3FD200006F0CAFC002398429E
:1038200005D0FA78552A02D0332A00D092E03360CE
:1038300007F04AFFFFF760FE1F22012400214F4BD3
:1038400010AE1A704E4B1C704E4B19704E4B1968CF
:103850009143163A0A431A60602219689143403A2C
:103860000A431A6008F000F907F0C6FEC120FF21E4
:10387000464B80001A588A431A50C5229200985825
:103880008843BF39014399509858414908408021E5
:10389000C9010143802099509958C0050902090ABD
:1038A0000143995080213B48490107F0BDFF0323A4
:1038B0002200394901940093384808F02DF92C2250
:1038C000374905A808F000F905AC61782078023482
:1038D00006F08EFCA642F8D1324C334B226803200E
:1038E0001A40A023DB0213432360802322689B0439
:1038F0001343236022682D4B1A4080239B031343FC
:1039000023602B4A2B4B934200D8012007F0FCFF89
:1039100007F02AFE80232268DB0413432360287803
:1039200008F082F8039B1878C0B207F0B5FE07F0E4
:1039300053FF2149042008F037F806F073FE00F029
:10394000A9F800F0E9FD00F091FE00F00BFA00206C
:1039500011B0F0BD00932100174A042007F004FFC6
:103960008023DB059C62FFF771FD61E74A0AFF1FB8
:1039700034F000409C3EFF1F385CFF1F480AFF1FC9
:10398000490AFF1F680AFF1FBCF0004000E100E089
:10399000FF00FFFFA03EFF1F2451FF1FA04EFF1F8F
:1039A000B8BB001114F00040FF7FF8FFFFFF9FFF3E
:1039B0000080FF1F9069FF1F3B00010870B50025C4
:1039C0002549264A26484D6308CA1B051B0DED18DC
:1039D0008242F9D100268022224B92058B63092175
:1039E000214B224C1E62224B1120DA67214BDA68F0
:1039F0008A43DA609A6820490A409A60266007F094
:103A0000A3FF112008F0D0F8636C1C4A13406364D4
:103A1000EE24E4006C431A4A200C04006423904214
:103A20000AD8FA223300D200904205D9154B0A2158
:103A3000C01807F0C9FFC3B2134A11201372D48013
:103A400008F082F8114B1B78002B04D1104B102189
:103A5000187807F0D9FD70BD000005400806054044
:103A600080060540FF01000000F0004000380040E3
:103A700004E100E03CF00040FFDFFFFFFFFEFFFF3E
:103A8000B70B000030F8FFFF205CFF1F5A5EFF1FDE
:103A9000585CFF1F002210B51100112007F074FEC2
:103AA00010BD0000F8B500230926364F364C3B62A6
:103AB000E3681120B343E36008F076F8112007F0C3
:103AC00043FF112007F010FF402322681025134305
:103AD000236080236268DB02134363608023A26853
:103AE00002211343A360A368284A08201340A3605F
:103AF0008023A2689B0113430122A360236CAB4384
:103B00002364236C1343236480231B013B62226BD9
:103B10001F4B1A402263626B1A406263A26B1A4009
:103B2000A263E26B1340E363E3681A4A1340E36065
:103B300006F05EFB0121082006F06EFC8023164A89
:103B40005B00516C11200B43536407F04DFDFD21C8
:103B5000C720124B124A89005A50A36B80002B4396
:103B6000A363E3680F4A3343E3600F4B19581140D6
:103B7000802212020A431A50802292051A600B4BCF
:103B80005D63F8BD00F000403CF00040FFFFDFFF48
:103B9000EFFFEFFFFFFF7FFF003800400000FF1F37
:103BA000BD390011FF00FFFF00E100E0000005400B
:103BB00030B503A804880B20002C0ED14968074DAE
:103BC00008784978090201430A20A94205D1012158
:103BD00020001980024B1B7A137030BD192A000097
:103BE000205CFF1FF7B5150008AA16884A680F4F1A
:103BF00014785278120222430A24BA4214D10122C4
:103C0000DBB2019200962A0007F046FC041E0BD19D
:103C1000074B1B68002B07D068782A7800021043F6
:103C200042425041013098472000FEBD0229000069
:103C3000A45BFF1F30B5012503790400BFB02B4200
:103C400011D00A49408806F093FF28420BD0084B58
:103C500001A95B8D4D800B80064B00221B7A60888A
:103C60000B7104F08DF83FB030BDC0469C5BFF1F68
:103C7000D83AFF1F205CFF1F10B50549054806F024
:103C80002DFF0421044A054806F0EAFE10BDC04697
:103C90009C5BFF1FFFFF0000E4BB0011D83AFF1F31
:103CA00010B5024804F0EEFE10BDC046353C0011D0
:103CB000062310B5837010330371443B43712A33DC
:103CC00083714433C37100230222012103720E4B1E
:103CD000027041701C8881724472197A0273C17239
:103CE0009A784273DA7882730322C2731A79027463
:103CF0005A7942740C2282749A79C274DB79037502
:103D00001123C370152010BD205CFF1F10B51420B7
:103D100007F09AFE124B14220021186007F02CFFC6
:103D2000002007F039FE012007F0F6FC022007F022
:103D30009BFC032004F04AF9042006F05FF90520FB
:103D400003F088FB062004F055F8072001F052FA32
:103D5000082006F065FE092001F03AF810BDC046C3
:103D6000A85BFF1F07F070FC012007F0BDFC07F007
:103D70000BFC0000094B10B50400984205D0012946
:103D800004D12000064906F0A9FE10BD0229FCD18D
:103D9000013904F035FE0028F3D0F6E7FEFF0000FD
:103DA000CE5BFF1F70B50D7A100004AA2C00168898
:103DB00010221440154220D1002E20D10A78022A68
:103DC00018D14A68517815780E4A09022943914260
:103DD00005D00D4A914209D01C800A2404E0142227
:103DE0000A491A8007F070FE200070BD0C220849B5
:103DF0001A80F7E71C800124F6E70824F4E70B2477
:103E0000F2E7C046F3FF0000F4FF00002C3DFF1F67
:103E1000C0BC001110B504000749084806F05EFE5A
:103E2000074804F06FFD0020E40704D50721054A88
:103E3000054806F015FE10BDCE5BFF1FFFFF00001A
:103E4000753D001128BC00111C3BFF1F00B50C4B39
:103E5000BFB01A780B4902A800F0C2FC6B4680B2D2
:103E6000D880002809D06A46074B01A91B88938097
:103E7000064B0022188803F083FF3FB000BDC04608
:103E8000AC5BFF1FAD5BFF1F763BFF1F803CFF1F3E
:103E900000B50C4BBFB01A780B4902A801F0B6FE72
:103EA0006B4680B2D880002809D06A46074B01A92A
:103EB0005B8D9380064B0022188803F061FF3FB0B2
:103EC00000BDC046D65BFF1FD75BFF1F1C3BFF1F1B
:103ED000803CFF1FF7B50E00377A1C0008AB1100BD
:103EE0003D001A8820231D401F423CD13378022B0D
:103EF0003BD173681F785B781B023B431E4FBB426C
:103F000008D01E4FBB4214D01D4DAB4221D00A2514
:103F10002800FEBD002A2AD1142C2AD82200F068DD
:103F200007F0D2FD174B1C70012CF1D9FFF7B0FF41
:103F3000EEE7002A1BD1202C1BD82200F06807F0E6
:103F4000C3FD114B04211C70104B187807F05CFB6B
:103F5000DEE7E3B20124009201940A00310007F089
:103F60009BFA0500D4E70825D2E70125D0E70B2509
:103F7000CEE70D25CCE7C046F3FF0000F4FF0000BC
:103F800002290000D65BFF1FAC5BFF1F585CFF1FC0
:103F9000332310B5040003700A220749013007F0EB
:103FA00093FD064B0F201B681A0AE37222731A0C4A
:103FB0001B0E6273A37310BD205CFF1F485CFF1FC4
:103FC00030B5012503790400BFB02B4213D00B4953
:103FD000408806F0CDFD28420DD06A46084B02A865
:103FE0001B889380FFF7D4FF6B46D880002260883F
:103FF00001A903F0C5FE3FB030BDC046CE5BFF1F38
:10400000763BFF1F10B5024804F03CFD10BDC046D2
:10401000C13F001170B5160004AA148805AA1578CE
:104020004A685078117800022A4A08438018052807
:104030004BD807F069FB03131E29343F0720032CDC
:104040000BD80422121BAA4200D92A0022491A8046
:104050003000091907F038FD002070BD0720112C31
:10406000FBD81222121BAA4200D92A001B491A802F
:10407000EEE707200E2CF0D80F22121BAA4200D91F
:104080002A0017491A80E3E70720032CE5D8042209
:10409000121BAA4200D92A0012491A80D8E7072029
:1040A000032CDAD80422121BAA4200D92A000E4996
:1040B0001A80CDE70720032CCFD80422121BAA4276
:1040C00000D92A0009491A80C2E700220A201A8072
:1040D000C3E7C046DCD5FFFF73BC0011F45BFF1FD4
:1040E00063BC00115EBC001159BC001154BC00112E
:1040F00010B50D21024A034806F0B2FC10BDC046BF
:1041000048BC00118C3BFF1FF0B50024274E85B042
:104110003000B47100F0E2F8254D264BEA89297C85
:104120009A422FD10423300003AA00F057F904006B
:10413000300000F011F90123B371002C34D16B462B
:1041400099892B68C9BA4B4329891B4A1B145B18F0
:1041500053806B46D9896B6849BA89B24B436989E8
:104160001B0C5B181548191C1BB2834200DD011C97
:104170000B0400D5002113889180013313802000A7
:1041800005B0F0BD0227220003AB3000009700F01D
:10419000F7F80E230400297C0122300000976B44BD
:1041A00000F0EEF80443C3E71C00E8E7643CFF1F9F
:1041B000085CFF1F83050000205CFF1F0F27000025
:1041C00073B5234E300000F089F8224D07236A466C
:1041D0003000297C00F002F904003000002C33D1BB
:1041E0006B461B787F2B2FD800F0B6F86B46D8783B
:1041F000F02302041B031A406B469B8816495BBAE6
:104200009BB21A432B68000953432A891B0C9B1845
:104210004B806B465A789B7812031B011A436B68DC
:10422000024353436A891B0C9B180C481A1C1BB28F
:10423000834200DD021C130400D500220B888A8013
:1042400001330B80200076BD00F086F80124F9E7E9
:10425000643CFF1F085CFF1F205CFF1F0F2700004E
:1042600070B5114C237C002B0FD0382B0ED10F4D85
:10427000280000F033F8CC23AC222800217C9B01DD
:1042800000F0F4F8280000F067F870BD084BE289F0
:104290009A42FAD1054D280000F020F800222800AB
:1042A000217C00F0C5F8EDE7085CFF1F643CFF1FB0
:1042B0008305000010B5084B1A7C002A09D05B6901
:1042C000002B06D09847041E01D0FEF799FE20006F
:1042D00010BD0124F9E7C046085CFF1F70B5C17925
:1042E00005000C00631E9C411A4BE402E4184900CF
:1042F0000460C9B2007906F0C5F8E9796879490027
:104300000131C9B206F0BEF8E8790930C0B207F051
:10431000EBFA0023E36661332360AA795B3B002A52
:104320000ED022689A43023B134323600A23E361C1
:104330000733236200232363A3630133E36370BD68
:1043400022689A43022313432360462363610633A2
:10435000A361EFE70050004070B50025040003683A
:10436000DD66C0790930C0B207F01EFC2900207953
:1043700006F024F82900607906F020F870BD0000EE
:10438000F8B51E0006AB1D78002304681700E3662D
:10439000616007F0F1F801238022E3662B002761BA
:1043A0005200013B08D207F0D7FA08200A4A1168E8
:1043B000002D03D12800F8BD2261F2E7236F0342EC
:1043C00003D02369013D3370013613685B1A032B58
:1043D000EED90125EEE7C0466008FF1F70B51C004E
:1043E000002305681600EB66696007F0C5F8012335
:1043F0008022EB6623005200013B08D207F0ACFAA2
:1044000008200A4A1168002C03D1200070BD2A61DF
:10441000F2E72B6F034203D02B69013C3370013666
:1044200013685B1A032BEED90124EEE76008FF1F27
:10443000002370B504681500E366616007F09CF81E
:104440000123E366256107F087FA8020064A800091
:104450001168636B034205D113685B1A032BF8D90B
:10446000012070BD0020FCE76008FF1F70B51D0033
:10447000002304681600E366616007F07DF80123FD
:10448000E36626610F33626B1A42FCD02B0A23616C
:104490001023626B1A42FCD0EDB2256107F05CFA82
:1044A0008020074A80001168636B034205D11368BE
:1044B0005B1A032BF8D9012070BD0020FCE7C04631
:1044C0006008FF1F70B51E00002305681400EB662E
:1044D000696007F051F80123A619EB660F33B44267
:1044E0000ED107F039FA80200A4A800011686B6B00
:1044F00003420CD113685B1A032BF8D9012070BD5D
:1045000021782961696B1942FCD00134E7E700206A
:10451000F5E7C0466008FF1F10B5084CE368002BA4
:1045200008D18022064B52021B689B186360054B22
:104530001B68236007F000FAA06010BD485CFF1FF5
:10454000C8F00040CCF0004070B5184A936A916AF8
:104550009942FBD116498A689A421FD39A1A8B60F6
:10456000144B0126186893B2D202D20E4343424341
:1045700000204C681B0A1B1912029B180E4C0A687B
:104580004B60551CA3420CD8002801D04B600A6038
:104590000A4A136008680A4B186070BD581E821AD8
:1045A000DDE7084A30009B182A00EAE700F00040E7
:1045B000485CFF1F140AFF1F40420F00C8F0004074
:1045C000CCF00040C0BDF0FF70B51F4C23793F2BED
:1045D00001D93F2323711D4B22791A701878C0B27C
:1045E00007F0AAF818231A491A4A0B801A491380AF
:1045F0000B805380A379194980200B800C21938074
:1046000001334B43164D191C0001834200D9011C94
:104610002980D1806379002B11D101336371237A12
:10462000012B01D8022323726279237A0D48534368
:104630000A21584307F0C8F90B4D286070BDA02B24
:10464000EDD9A023EAE7C0463C5CFF1F480AFF1FE4
:104650007E3CFF1F483EFF1F7C3CFF1F7A3CFF1F34
:10466000783CFF1F710200002C5CFF1FF8B514217D
:104670000020FEF7B3FE114C011E114D09D10C2292
:10468000104BC1CBC1C4280007F076FAFFF79CFF9E
:10469000F8BD0C2220000C49FEF774FE0C2802D055
:1046A000084B43CB43C40C2228000849FEF76AFE9E
:1046B0000C28EBD00C220021E5E7C0463C5CFF1F34
:1046C000085CFF1FB4BC0011FC0C0000F50C0000DE
:1046D000F0B51D4C8022A544040088206946520193
:1046E000400507F0C9F9902212016A441300200026
:1046F00032C832C316C816C38023144C144FA668A0
:104700009B033343A3603B6007F086F98823A068CE
:104710005B05C01807F030F90025882329008022A6
:10472000A0685B05C01840196944520007F0FCF905
:1047300080230135FF355B019D42EED1A6603E60CE
:10474000044B9D44F0BDC046FCEFFFFFBC3DFF1F86
:104750009808FF1F04100000F0B5040087B000287F
:1047600025D0684607F000F91B4C022806D1062226
:104770006946200007F060F8002816D0694600233B
:1047800001250F262F00E25C01331009103087400D
:1047900038002F00324097403A0002434A61043902
:1047A000062BEFD16846FFF793FF07B0F0BD182244
:1047B00069460A4807F060F96A46A300D3580133F6
:1047C00005D01822FF21684607F0D6F9EAE7013440
:1047D000062CF1D1E9E7C0466509FF1F0009001169
:1047E000F0B5002504000E0085B0AA4200D186E095
:1047F0004B1C087801934B78897837790902194363
:10480000F3783F061B040B431F430397207065702A
:10481000252800D196E033D8112813D806F0C4FE1D
:1048200069002B012B012B012B01AA00B800B1005C
:104830002B012B012B012B012B012B012B012B0118
:1048400005012501232800D1DEE0DB2800D034E17A
:10485000042A00D8ACE01025052A05D0551F2A00EF
:104860003800711D07F030F905223100200007F0F3
:104870002BF92A003900601D07F026F905353EE0C6
:10488000562859D010D8332800D19DE0552839D06A
:104890002628DAD19F4B2900132218001D0007F0AB
:1048A0006BF9FEF7ADFB5CE0712800D177E0722870
:1048B00000D180E0602800D18BE0DC28C5D1022A3D
:1048C00000D875E07378BFB26370B378A370032A21
:1048D00005D0033A390092B2F01CFEF78DFC10228D
:1048E0003900E01CFEF74EFDC51C002807DA607099
:1048F0005CE00C222000884907F0E6F80C2528002F
:1049000005B0F0BD013A854D0C2A13D8002A0AD013
:104910002800019907F0D8F8FFF756FE0C2228006E
:104920007F49FEF769FC29000C22601C07F0CCF8D7
:104930000D25E4E70C22EBE7784D7A4B2A0043CBB8
:1049400043C2E9E7013A734D0C2A11D8002A08D076
:104950000199280007F0B8F80C2228007249FEF7E8
:104960004BFC29001322601C07F0AEF81425C6E7A3
:104970000C22EDE705226D49601C07F0A5F806251D
:10498000BDE712226A49601C07F09EF81325B6E7BE
:1049900008226849601C07F097F80925AFE771788D
:1049A000F02905D8644B188801F08CFD0225A6E794
:1049B000FF236370FAE7614B012A03D072789A7083
:1049C0006270F3E79B78F4E72000FFF7E1FA050057
:1049D00095E7013A594B5A4D072A10D8002A10D0B2
:1049E000012128005970019907F06EF801F048F88C
:1049F00029000722601C07F067F808257FE70722D7
:104A0000EEE700225A70F3E7042A04D94D4D2F60D7
:104A100006F092FFA860FFF797FD0422039003A918
:104A2000601C07F051F8052569E7474D062A15D99E
:104A300006222800019906F0FFFE00280ED006226B
:104A40000199280007F040F8062240492800FEF7A7
:104A5000D3FB0123394A91780B4393702900062236
:104A6000601C07F031F8072549E7012AA0D07078CB
:104A7000FFF772FE9AE7012800D0E6E6931E344F56
:104A80001A2B04D87378002B09D100F015F9314B9B
:104A900039001D78601C6A1E07F016F82FE7551EB6
:104AA0002A000199380007F00FF82B49AAB2380004
:104AB000FEF7A2FB00F036F9E9E7DA281DD1042A57
:104AC00000D875E7082A15D9B37972791B02134308
:104AD000F27912041A43337A1B0613433B603B6896
:104AE000052231002000039306F0EEFF0422601D32
:104AF00003A950E7FE236370F1E7DE2800D057E7F3
:104B0000511E012A01D10025F9E6019800F09EFF0F
:104B1000F9E7C046085CFF1FC0BC00113C5CFF1FEA
:104B2000FC0C0000B4BC0011F50C0000145CFF1F6D
:104B3000F45BFF1FC03DFF1F803CFF1F385CFF1F61
:104B40001D3DFF1F485CFF1F6509FF1FADAC000046
:104B5000395EFF1F375EFF1FAEDE000070477047F3
:104B6000020010B5094B0A32094C92B2DA815A821E
:104B700098811882207802F00BFB0422054B01215A
:104B800020781A7006F040FD10BDC0464A3DFF1F58
:104B9000825EFF1F815EFF1F013870B5042809D8AF
:104BA00006F0B2FD030928081200234B02211878F1
:104BB00006F02AFD70BD204B0821187806F064FD30
:104BC00000221E4B1A72F5E7802200241B4B1A4D5F
:104BD00052001A8108211A682878DC7206F04CFD10
:104BE0002100287806F020FD012000F04FFE00F0A3
:104BF00047FFDFE7104B0821187806F045FD104805
:104C0000FFF756F80F4B104A9B79002093800F4A0C
:104C100013808022094B5200D8721A8100F036FEB0
:104C200000F02EFF0A4B9B78002BC3D0094A13607B
:104C300006F0DAFDBEE7C046585CFF1F2C5CFF1F84
:104C4000893CFF1F3C5CFF1F483EFF1F7A3CFF1F53
:104C5000385CFF1F34F0004010B501290BD101284A
:104C600009D1054B1B78002B05D02622034B0448A5
:104C70005A72FFF775FF10BD5A5EFF1F2C5CFF1FB5
:104C8000C40900000300F0B50A4D8E18B14202D1EC
:104C900052008018F0BD0C782F6824093C5D0F2766
:104CA0001C700C7801313C402F683C5D5C70023315
:104CB000ECE7C046743CFF1F0D22114B10B51A7073
:104CC0000C23104C10492370093A033B0F486370C2
:104CD00006F0FAFE2D2301220D490E48A371FFF7BD
:104CE000D1FF01220C49FFF7CDFF01220B49FFF74D
:104CF000C9FF00220A491000FEF77EFA10BDC04627
:104D0000565EFF1F375EFF1F73BC0011395EFF1F29
:104D10006709FF1F3E5EFF1F6609FF1F6509FF1F32
:104D2000AEDE000070B5124C132220001149FEF7D0
:104D300029FB114D002817DDAB78002B14D0431C44
:104D40002B7009236B700023001903702878290049
:104D50000130C0B206F060FD297822000139C9B2E5
:104D6000002005F09BFD70BDFFF7A6FFEEE7C046F3
:104D7000395EFF1FAEDE0000375EFF1F10B5114B1E
:104D80001A781870002A0ED000280BD10E4B1A7812
:104D9000062A07D85423D340DB0703D50B4B1878DA
:104DA00002F0F6F910BD0028FCD0074B1B78012B50
:104DB00002D0033B022BF5D8044B0121187806F0F2
:104DC00023FCEFE75A5EFF1F815EFF1F825EFF1F1D
:104DD00070B54A4E4A4A4B493070012005F000FC3C
:104DE00000F0B2FEFEF70CF906F086FE03224649FB
:104DF0004648FFF747FF2D24030004221C70444956
:104E00000130FFF73FFF30230470424D424C4370A6
:104E100083702E3B062220004049EB87FEF7B2FA52
:104E2000062813D0200006F09FFD022809D0032198
:104E3000200006F051FE8D23E3706E3B2371193381
:104E40006371062220003549FEF7D6F9344B1B6802
:104E5000FC335C64FFF766FF0020FFF78FFF314CE7
:104E6000314A0121314B1278207802F053F9304A4F
:104E7000304B12780021207802F04CF901222E4BA1
:104E80001A702E4BDB78552B31D12D4B3B325A7299
:104E90002C4B2D4AAB81EA812B826A82202130780B
:104EA00006F08AFB0120404205F044FD012040420B
:104EB00005F0E0FDFFF71CF9FEF7DEFE00F0A4FCB4
:104EC00001204042FEF7A6FF012006F015FCF0206D
:104ED00001F0DCFA0121307806F096FB307802F020
:104EE000B3FA1A4806F0B8FCFEF7DCFD70BD642288
:104EF000174B5B7953431A000A32CBE7585CFF1F0C
:104F00005D4B0011594C0011C03DFF1FF45BFF1FAA
:104F1000145CFF1F4A3DFF1F6509FF1FADAC000079
:104F2000AC5EFF1F825EFF1FA83CFF1F893CFF1F76
:104F3000565EFF1F375EFF1F285EFF1F385CFF1F96
:104F40002C5CFF1FC4090000CE0900005A5CFF1F43
:104F50003C5CFF1FF8B50A0020230D001A401942DF
:104F600057D0574B1B78002B50D0FFF7EDFA554B1D
:104F7000554C564E99686268737A8A1ADB039A42D6
:104F800002D36160FEF78EFD327A217A531EDBB2C6
:104F9000994205D1FFF764F9002000F0A7FD0FE06A
:104FA0009142F9D300232372FFF784F9012000F026
:104FB0009DFD474F3800FEF77BFE390006F03CFBB5
:104FC000637A002B1FD0013BDBB26372002B1AD136
:104FD000404BDB78552B01D106F006FCE37A002B21
:104FE0000CD000233C4A3A4FE37213883800013357
:104FF0001380FEF75DFE390006F01EFB6423707916
:105000005843FFF7ADFD237A013323722020684017
:10501000F8BD0BB2002B0ADA304B187806F044FDCD
:10502000002801D006F0C8FC80200002EFE702242F
:10503000214206D0244B01201A72FFF79FFE200068
:10504000E5E70B071ED5FFF77FFA1E4B1E491F4CE5
:1050500098684A68637A821ADB039A4202D34860EE
:10506000FEF720FDFFF726F9FFF7FAF8012000F020
:105070003DFD00F0E3FB2368DB0701D5FEF7C2FF2F
:105080000820C4E71024214206D00D4B1B78002BCA
:10509000D5D1FEF705FED2E70124214207D0104802
:1050A00000F06CF806F078FB00F006FDC7E704247A
:1050B000080020402142ABD0FEF7C8FEBFE7C04643
:1050C0005A5EFF1F485CFF1F2C5CFF1F3C5CFF1FEC
:1050D000893CFF1F385CFF1F205CFF1F585CFF1FCF
:1050E0006C3CFF1FF0B51B4B1B4F1B883A8804001C
:1050F0001A4E1B4D85B09A420DD832889A420AD377
:10510000184B1A882B889A4205D1174A174B1288D8
:105110001B889A421BD0052001F00EFA3B8802AA98
:1051200013803388019053802B88114D93800F4B4F
:1051300002A91B88D3800F4B2A78188802F02AFF17
:105140000D4B08212878019A1C7006F0E5FB05B08C
:10515000F0BDC046265EFF1F7E3CFF1F7C3CFF1F4C
:105160007A3CFF1F245EFF1F225EFF1F783CFF1F5B
:10517000825EFF1F803CFF1F205EFF1F13B50C4B9C
:105180001C78002C11D1002801D00A4B18600A4A63
:105190000A4B11780A4A10780A4A01920A4A009288
:1051A000002205F073FA200016BD1124FBE7C0466B
:1051B000815EFF1F1C5EFF1F805EFF1F705EFF1F72
:1051C000825EFF1F5C5EFF1F605EFF1F10B5064B17
:1051D00012201B78052B06D1044B13221988044B8F
:1051E000187801F085FB10BD815EFF1F803CFF1F1A
:1051F000825EFF1F10B500240122114B524218702D
:10520000104B1C70104B1A8002F01EF904220F4B39
:1052100021001A700E480C3206F0F6FB1022210015
:105220000C4806F0F1FB07220B4B1C600B4B1C706B
:105230000B4B1C700B4B1A700B4B1C7010BDC046F7
:10524000825EFF1F815EFF1F803CFF1F805EFF1F8D
:10525000705EFF1F605EFF1F5C5EFF1F365EFF1FFC
:10526000355EFF1F823CFF1F345EFF1FF8B5174CF1
:105270000600257806A814240078052D23D1B41F34
:10528000134FA5B21824BD421DD88D1FADB2BD422B
:1052900019D8FA256D00AA4215D21D000D4F0A3DFE
:1052A000ADB2BD420FD80C4C26800C4C21800C496D
:1052B00000240A800B4A1380FFF714FF0A4B0421D5
:1052C000187806F0E1F92000F8BDC046815EFF1FA6
:1052D000790C0000750C00007E3CFF1F7C3CFF1F1A
:1052E0007A3CFF1F783CFF1F825EFF1FF0B50BB2B8
:1052F0000D0089B0002B00DB70E1A44E307806F081
:10530000D3FB041E50D00378A22B00D122E1D02B76
:105310001AD0912B45D143780E2B42D19C4B8288D9
:105320009A423ED19B4A83681278052A39D10320DC
:1053300018567F2835D0984B1B68002B31D05B68FE
:10534000002B2ED098472CE08078072829D806F02B
:10535000DBF90428183F3F74A8D86378002B0CD1E0
:1053600001218C4B19708D4B1A78002A5BD08C4B25
:10537000307801F0CFFE002855D00722854B1A70F7
:1053800051E061780029F8D1E378002B11D0854AEB
:10539000854B1278307801F0BDFE60706378002B89
:1053A000EBD1200006F008FB80200002684009B025
:1053B000F0BD784B1B78022BF3D00121307806F03A
:1053C0002BF90028EAD10121307806F01DF9E5E734
:1053D0006378002BD1D16F4F032807D13B78052B81
:1053E00002D101333B701EE00223FBE76F4B1A88AA
:1053F0006F4B0293002A0BD01B78002B03D00121A6
:10540000307806F089FA3B78062B04D1013BE9E7B6
:10541000029B1A70F7E7042B41D10121029B3078DF
:10542000197006F0F1F85C4B1B68002BB9D01B68B3
:10543000002BB6D0574A107884E76378554F002B7D
:1054400027D10622211D5B4806F03EFB62895A4B9C
:105450005A491A80A2895A4B1A80E3890B80052188
:10546000397058490A80584A1380228A574B1A804B
:10547000574B1B78012B09D11F2001F05DF8FA2250
:10548000920042430421307806F046FA0022484B4D
:1054900075E7312B00D070E70022454B1A700323CB
:1054A000A0E706220021434806F0AEFA0023454A51
:1054B00004211380444A30781380444A138006F054
:1054C000E3F80821307806F0DFF8A379083B5A4268
:1054D0005341304A03331370304B1B78002B06D0F6
:1054E000334B30781A78002A06D001F051FE0122A1
:1054F000314B52421A8096E70121197006F084F868
:10550000F5E70821307806F0BFF86378002B00D06B
:1055100047E72C4B2D4F0293E388029A0421138016
:10552000294B307803932389039A138063893B8046
:1055300006F072F8002800D033E7264B1B68002BDA
:1055400000D12EE7039902983A88098800881B68E1
:10555000984726E74379132B00D022E70389012BD4
:105560000AD11D4B1B78022B06D10821307806F09A
:105570008BF8FFF72BFE14E7052000F0DDFF082174
:105580000200307806F0C8F90BE7C046825EFF1FC4
:1055900005140000815EFF1F1C5EFF1FA83CFF1F5B
:1055A000893CFF1F565EFF1F375EFF1F585EFF1FBF
:1055B0005A5EFF1F295EFF1F803CFF1F305EFF1FEA
:1055C000325EFF1F265EFF1F245EFF1F225EFF1F4D
:1055D000285EFF1F185EFF1F205EFF1F8020C00196
:1055E000014200D0E2E6CB0731D5324B1B78002BCD
:1055F0001DD0314E05AC3378052B1AD1023B2370F8
:105600002E4B21001B7823722D4B1B7863722D4B80
:10561000187801F023FD002809D007202A4B3070AC
:105620001B68002B03D01B68002B00D0984701207B
:10563000BCE60E20254B06221B7825492370254BFE
:105640001B78637002ABC01806F03EFAD8E702235D
:1056500008001840194209D0174B1B78052B03D1BD
:105660001D4B188806F028FA02209FE604242142E8
:1056700003D0FFF737FD200098E608230800184004
:10568000194200D193E6154B1C78012C03D0022C53
:105690000DD008208AE6124B124A134913481B8882
:1056A0001288098800880094FFF7E0FDF1E7FFF712
:1056B0008DFDEEE75A5EFF1F815EFF1F823CFF1FDC
:1056C000345EFF1F825EFF1F1C5EFF1F365EFF1FE2
:1056D000833CFF1F355EFF1F803CFF1F205EFF1FC6
:1056E000783CFF1F7A3CFF1F7C3CFF1F7E3CFF1F66
:1056F00010B502A804880B20002C10D14968087846
:105700004978090201430C48814209D102211980DC
:105710000A4B59881170DB7800205BB2537010BDC2
:10572000074C0A20A142FAD102211980034B998823
:1057300011705B79F0E7C0466E2A0000205CFF1F05
:105740006F2A0000F7B5150008AA16884A680F4F9F
:1057500014785278120222430A24BA4214D1012248
:10576000DBB2019200962A0005F096FE041E0BD1D2
:10577000074B1B68002B07D068782A78000210437B
:1057800042425041013098472000FEBD02290000EE
:10579000945EFF1F30B5012503790400BFB02B4292
:1057A00025D01449408805F0E3F928420CD0124B6B
:1057B00001A95B8D00220B8002234B800F4B5B887D
:1057C0008B80608802F0DCFA0D49608805F0D0F922
:1057D000C0070CD50B4B01A91B8800220B800223AC
:1057E0004B80064B9B888B80608802F0C9FA3FB0E3
:1057F00030BDC0468C5EFF1FAC3CFF1F205CFF1F0E
:10580000845EFF1F063DFF1F10B5074C07492000AF
:1058100005F064F92000064905F060F90721054A02
:10582000054805F01DF910BDFFFF00008C5EFF1F4D
:10583000845EFF1FE0BC0011AC3CFF1F10B50248A6
:1058400003F020F910BDC04695570011022143080E
:1058500088400B400A31084003430E20024AD178A9
:1058600081430B43D37070471D3DFF1F064A1379D8
:10587000410705D580210B4380011371907170475A
:105880007F210B40F8E7C0461D3DFF1F054A5378B6
:10589000002803D080210B43537070477F210B40B9
:1058A000FAE7C0461D3DFF1F0F21114BDA780A4071
:1058B000DA70502810D901310A43DA702022D978E1
:1058C0000A43DA704022D9780A43DA708022D97804
:1058D00052420A43DA7005E03C28EFD82828F1D874
:1058E0001428F3D80122D9780A43DA707047C046E9
:1058F0001D3DFF1FF8B57F23324D04006E789E4397
:10590000314B984205DD76232B70363B33436B7069
:10591000F8BD2E4B984203DA58232B701433F5E769
:1059200083B21A0000215F32294892B2294F2970B0
:1059300082422DD9A9708C4203DA5B421CB220232B
:105940002B70053420B20A2106F03EF804B2FA2387
:105950009B009C4233DB80232A785B4213432B70ED
:105960006421200006F030F80A2100B205F014FE90
:1059700009B22A787B5C13432B700A21200006F0C1
:1059800023F80A2100B205F007FE09B27B5C0AE0A9
:105990008022AA70002CDADA5B421CB220232B7022
:1059A0005F23092CE9DC1E430A2120006E7005F0FC
:1059B000F3FD09B2AA787B5C1343AB70A8E7632CB4
:1059C000CEDCEDE71D3DFF1F1B4E00001DFCFFFF61
:1059D0002A0800000ABD00117F23F7B5194FCD0139
:1059E0003E7904009E433E71EDB2632806DD093B1B
:1059F00033433B7140231D437D71F7BD03000933E1
:105A000004DA582333433B716C23F4E70E4B0193C4
:105A100000280BDA0423444224B23B710A212000FF
:105A200005F0BAFD019B09B25B5CE4E70928F5DDEE
:105A30000A2105F0C9FF019B00B21B5C1E433E71A9
:105A4000ECE7C0461D3DFF1F0ABD0011F8B50A4F27
:105A500005003B780E00002B0CD0084C2000FEF710
:105A60003DFC33002A0020003978FEF72BFD200092
:105A7000FEF772FCF8BDC046A05EFF1F243DFF1F6D
:105A800070B50A4E0A4D07223100280005F0D4FEF9
:105A9000002809D0074C31000722280006F014F82E
:105AA00008212000FFF7D2FF70BDC0461D3DFF1F3B
:105AB000995EFF1F985EFF1F7F2210B50A4B597831
:105AC0009143033A1A70103A0A435A7078220E2111
:105AD0009A70DA788A43DA7006221A7130325A7173
:105AE000FFF7CEFF10BDC0461D3DFF1F10B50028BB
:105AF00024D0134C0A210223E05E05F065FF00B2BA
:105B0000FFF7F8FE0423E05E642105F05DFF01214C
:105B100000B2FFF761FF207AFFF7C6FE0320FFF710
:105B200095FE0020FFF7A2FE064B18780538434289
:105B30005841C0B2FFF7AAFEFFF7A2FF10BDC04652
:105B4000205CFF1F815EFF1F70B50024094D2800F7
:105B5000AC71FEF7C3FB10233E212800064AFEF776
:105B6000B1FCA04200D13E34044B28001C70FEF76B
:105B7000F3FB70BD243DFF1FFABC0011A05EFF1FA8
:105B80000200F0B501270A480A4E51188B1A002B63
:105B900000DCF0BD08241578430868403840400018
:105BA000805B013C58406D08002CF5D10132EDE7D7
:105BB000FFFF00001ABD0011F0B500250F269D4221
:105BC00000DBF0BD4C5D070944403440A400A05800
:105BD00001357840F3E70000F0B589B06A460D0062
:105BE0000B000F27110010351C7801332600240903
:105BF0003E40167054700232AB42F5D12023024A67
:105C0000FFF7DAFF09B0F0BD20BD0011F0B54E7806
:105C10000B7889B036020C00170001901E43012A50
:105C200061D9954B9E4200D877E001339E421CD14A
:105C3000062A17D1CA788B7812021A430B791B04F3
:105C400013434A7912061A438C4B5A6100221A7088
:105C50005A808B4A5A608B4A9A608B4ADA600020DD
:105C600009B0F0BD88225205EEE7884B9E423CD138
:105C700082498B78002B00D0F6E00C2A31D10F221C
:105C8000A3789343E2781202134322791204134358
:105C90006279120613434B60E279A0791202024343
:105CA000207A00041043627A12060243CA60E27A44
:105CB000A07A1202024376484A81834208D804231C
:105CC0006E49142201980B7005F0FEFE1420C7E700
:105CD0001201D21889235B059A42F0D801238B70F8
:105CE000BDE7022AFAD00523EAE76A4A0123964271
:105CF000E6D1FFF76BFA052F0CD9E378A2781B02E7
:105D00001343227912041A4363791B061343624A30
:105D10000393136005F068FDA1E7584D2B78002B25
:105D20009DD1AB78002B00D1A0E02B8901339BB231
:105D30000093B34200D091E0132AD4D9CF7C8B7C5E
:105D40003F02122120001F43FFF71AFF874200D0B5
:105D50008EE0002E3DD1E378A2781B021343227916
:105D6000E96812041A4363791B06134303930A225A
:105D70008B4212D1FF23A370E370237163716B898F
:105D8000002B09D1E37B227C1B0212041343A27B6C
:105D900013431B0901336B8100226B89002B8ED0CA
:105DA000002A67D1686837013818000B6B69000357
:105DB0000390984205D9686105F0DEFDEB78013368
:105DC000EB7068681022A11C381805F0ADFE2E811A
:105DD00045E76F89009A7B1E9BB293423AD1E278E5
:105DE000A37812021A43237905A81B04134362798E
:105DF0006C6812061A43EB6800920392211D0C2274
:105E0000049305F061FE0120260004A940421036EB
:105E1000FFF7E2FE013F012F17D1009A0B23286103
:105E2000824200D04CE704221C49200005F07CFE91
:105E3000042203A9686805F01FFEE968039AFF239E
:105E4000914200D13CE7F73B3AE73100FFF7C4FE4F
:105E50001036DFE70923B742A4D831E7009BB342ED
:105E600000D9FCE607232BE7022329E7032327E7D2
:105E7000062325E70A2323E7FFFE00002C3DFF1F32
:105E800000000111FFFF00005048593601FF0000DB
:105E9000FFFF001102FF000034F00040383DFF1FFB
:105EA00010B5034C0B000122210000F06BFA10BD6D
:105EB000616000110B8870B506000D000224162BDE
:105EC00011D92B000322094900F05CFA041E0AD103
:105ED000074B2A881B88191C934200D9111C3000DB
:105EE00089B200F0EFFA200070BDC0468D6000114D
:105EF000C65EFF1F10B54A780400013A0B0002206D
:105F0000012A07D80A78002A04D005222000024975
:105F100000F038FA10BDC046BB6000110A7810B519
:105F20000B0004000220002A04D0072220000249AE
:105F300000F028FA10BDC046676100110A7810B55C
:105F40000B0004000220002A04D00922200002498C
:105F500000F018FA10BDC046CD61001110B5034C19
:105F60000B000B22210000F00DFA10BDFD610011A5
:105F700010B5034C0B000D22210000F003FA10BDF8
:105F80006F62001110B5034C0B000F22210000F0CE
:105F9000F9F910BDC96200110A7810B50B000400B0
:105FA0000220002A04D011222000024900F0EAF960
:105FB00010BDC046D9620011002310B5132219008C
:105FC00000F0E0F910BD000010B5034C0B001722E3
:105FD000210000F0D7F910BD2B630011002310B58C
:105FE0001922190000F0CEF910BD000010B5034CC5
:105FF0000B001B22210000F0C5F910BD65630011E4
:10600000F7B584890D0006000121002C22D0002361
:106010008268D3561778002B1EDA0C2C1AD90C3C48
:10602000A4B2131940880093230002F086FE431E99
:10603000984101307B06DB0F6B703F23013C1F4012
:10604000A4B22870AF70AC80002C07D0B3680133C5
:10605000AB6000210800FEBD0020EBE7AC60F8E774
:106060000B7803704B8843704B881B0A83700B7945
:10607000C370042070470420022B06D100205378FF
:1060800011781B02009A0B43138070470B88037032
:106090000B881B0A4370022070470420009983423A
:1060A0000AD1537810781B0203430B80D378907881
:1060B0001B02034300204B807047F8B50D004B785E
:1060C00001240021461C03702B788B4201D820004C
:1060D000F8BD6B78B01C4F1C012B10D189006918DA
:1060E0004B88022233704B88B9001B0A7370691801
:1060F00005F04AFC04360434A4B2F9B2E4E71223F2
:1061000059436B185A88043132705B8810221B0A7D
:106110007370691805F038FC12361234ECE770B56C
:10612000049D14001E00052B01D8042070BD637867
:1061300012781B0213432B80E378A2781B021343CF
:1061400002226B802A71211D681D063E05F01CFC91
:10615000B2B22A81E92AE8D82800A11D0A3005F048
:1061600013FC0020E2E7002310B50A789A4201D818
:10617000900010BD9A008A18548801330470548826
:10618000DBB2240A4470948884709288120AC27028
:106190000430EAE710B51100029C062B04D004205D
:1061A0001022142B01D010BD022222714B780878E6
:1061B0001B0203432380CB7888781B020343638050
:1061C0000431601D05F0E0FB0020ECE710B50C7811
:1061D0008B7804315C43E4B203702200013005F097
:1061E000D3FB601C10BD0420022B06D10020537885
:1061F00011781B02009A0B431380704710B50C00F6
:106200000A88023105F0C0FB208810BD70B504007B
:106210000D0004981100012B01D8042070BD1678E0
:1062200052781202324302800200F132557014702B
:10623000E125002C00D10C35023B9AB24280AA42E3
:10624000EBD80231043005F09FFB0020E6E7042084
:10625000009983420AD1537810781B0203430B80C4
:10626000D37890781B02034300204B80704710B511
:106270000C000A88023105F087FB208810BD000061
:1062800070B501211E000420049C0E400B4218D161
:10629000CB40DDB28D4214D90A49DBB2098899425C
:1062A0000FD32300EE331D703300580011184978C6
:1062B000165C0902314301332152D9B28D42F4D820
:1062C000002070BD443DFF1F10B50C000A8802314C
:1062D00005F05AFB208810BD10B50C788B7804317E
:1062E0005C43E4B203702200013005F04DFB601CFA
:1062F00010BD10B511000298032B01D8042010BD69
:1063000014785278043B120222430280CA788C78B7
:106310001202224342809AB28280EB2AEED80431E4
:10632000063005F031FB0020E9E710B50C000B88C2
:1063300003700B881B0A43704B8883704B881B0AC1
:10634000C3708A880430063105F01EFBA088043033
:1063500080B210BD0420012B03D100201378009AD5
:106360001370704710B50C000B8803700B881B0A64
:1063700043704A880230043105F006FB6088023021
:1063800080B210BDF0B589B003931E4B029242005B
:106390000700D05A019102F020F81325061E2DD0D7
:1063A000029B01240370019B002B04D00019039968
:1063B0009847001984B26B461B7A5BB2002B0FDA48
:1063C0001021380002F01CFB1925002813D13000E1
:1063D0003219E1B202F066FC051E0CD10C34A4B2F5
:1063E000042304AA380005A993800696948101F03D
:1063F000AFFD051E02D0300005F0BEF9280009B03F
:10640000F0BDC046C45EFF1F70B505000C0000283B
:106410000CD00020814209D010222000044905F050
:10642000B3FA01202B7823736B78637370BDC04679
:1064300060BD0011F0B506000D0017001C0085B00E
:1064400002291BD00020102907D1022B07D0102BC6
:1064500003D115E00020102C08D005B0F0BD69462E
:106460003800FFF7D1FF2A0069460BE0694630008B
:10647000FFF7CAFF22006946380004E0022BE9D189
:106480002A003900300005F00FF9E6E7031CF02878
:1064900000D9F023032008499AB2013A0B80D317A0
:1064A000034006499B189B100B80D30F04499B188F
:1064B0005B100B807047C046483DFF1F463DFF1FE5
:1064C000443DFF1F034B1B888B4202D3024B40000D
:1064D000C1527047483DFF1FC45EFF1F014B400083
:1064E000185A7047C45EFF1F1722014B1A8070476D
:1064F000C45EFF1F70B505000E2005F0E5F9041E0F
:1065000013D0D023037000230622837007494570FF
:10651000033005F039FA064B2100DA8A62811B7ECE
:106520002373044B187805F02FFB70BDE05EFF1F4E
:10653000D05EFF1F983DFF1F262803D8024B400066
:10654000C05A70470148FCE74A3DFF1FFFFF0000AB
:1065500070B506000C00094D1C220021280005F032
:1065600053FA074B1E70074B1C7005F07DF9012391
:10657000002801D0002312202B7070BDD05EFF1FB9
:10658000983DFF1FF15EFF1F70B505000D4C080020
:10659000E260A16010220021656005F0E5FA0128A3
:1065A00003D11021A06802F058FD1022002128001C
:1065B00005F0DAFA012803D11021606802F04DFDE0
:1065C00070BDC046D05EFF1F70B5041E05D1002906
:1065D00003D006220D4805F0D7F90D4B1D78012D8B
:1065E00011D1002C05D102221A7005F00DF92800F6
:1065F00070BD00221A70074B1B78FF2BF7D02000CC
:10660000FFF778FFF3E70025F1E7C046E05EFF1FE4
:10661000D05EFF1F983DFF1F030010B5002801D179
:10662000002010BD00780B4A002803D15988D18280
:106630001B7913761378022BF2D10023984200D1F4
:1066400003331370044B1B78FF2B01D0FFF752FF6D
:106650000120E6E7D05EFF1F983DFF1F002911D003
:1066600000280CD04B79012803D140225242134319
:1066700003E03F221340032802D001204B717047F2
:106680004022F4E70800FAE770B5094D01002878C8
:1066900000280BD0074C0622200005F075F92100D8
:1066A0002878FFF7DBFF200005F076FA70BDC046C2
:1066B000F05EFF1FCA5EFF1F00290AD0012808D123
:1066C0003F224B799343C02B03D0403B5A42534166
:1066D000981C704770B5174D06002B78FF2B15D00E
:1066E0000A2005F0F1F8041E10D0D0230370C83B37
:1066F0008370114B11491B784670C3700622043019
:1067000005F042F92100287805F03EFA0C4B1B7881
:10671000012B0DD10B4B1B68002B03D09B68002B6A
:1067200000D09847084B04211878084A04F0A4FFC9
:1067300070BDC046983DFF1FF05EFF1FCA5EFF1F81
:10674000EC5EFF1F185FFF1F1C5FFF1F60EA000069
:10675000014B98687047C046D05EFF1F014BDB6855
:1067600018687047D05EFF1F074B10B5DA681368D2
:1067700001331360054B1878FF2803D08021C9012D
:1067800004F042FF10BDC046D05EFF1F983DFF1FC2
:10679000F7B50E0002F0C8F8051E1CD00E4B0662BD
:1067A0001F78002F00D10778AB791020019305F0F6
:1067B0008BF8041E0FD0D0230380C73B8370019B4E
:1067C000E91DC3700622043005F0DEF82100380010
:1067D000E66005F0D9F9F7BD963DFF1F014B18782B
:1067E0007047C046F05EFF1F054B002805D1054BE2
:1067F0001A78054B002A00D1014B18007047C0469B
:10680000E05EFF1FF05EFF1FCA5EFF1F014B58686E
:106810007047C046D05EFF1F024B1868431E984168
:10682000C0B27047F45EFF1F421E03000120152A0C
:1068300003D9FF3B5A425341D8B27047F0B51C0010
:1068400000230E0085B0039002920B70029A9342CF
:1068500001D3002019E0E55C5A1CD2B2002DF8D01B
:10686000029851198142F4DC0233DFB2A35C1800B4
:106870000193FFF7D9FF002807D0013D019A039942
:10688000EBB233708A4202D1E01905B0F0BDDB19DA
:10689000DBB2DBE710B50C0002F09EF8030012201B
:1068A000002B03D02100588805F0F6F810BD000039
:1068B00070B50E4D84006359002B15D0186A00285E
:1068C00001D004F041FF2B59586A002801D004F090
:1068D0003BFF2B59986A002801D004F035FF285956
:1068E00004F032FF00232B5170BDC046005FFF1F34
:1068F0001C4B70B504000E00150099420AD11A4BCA
:106900001B68002B01D1122070BD1B68002BFAD030
:106910009847F9E7154B994215D1134B1B68002B8B
:106920000AD01B68002B07D09847002804D1104BD1
:106930001C70104B1D70E7E729002000FFF7AAFF2D
:106940000028E1D1F3E7080001F0EEFF0028DAD0DB
:1069500003780320A342D7D12900300005F09CF82A
:10696000D2E7C046FEFF0000FC5EFF1FFFFF0000F5
:10697000F95EFF1FF85EFF1FF7B50400808801F085
:10698000D3FF0025A84203D00578A08802F008F8BC
:106990001C4E3378002B1FD0AB421DD11A4B280060
:1069A0001978FFF777FF002818D000233370A379F8
:1069B0000820A778A688019304F086FF011E0DD059
:1069C000D0230370CA3B8370019B4770868083711C
:1069D000280005F0D9F801E0002DE8D1A0880B4B84
:1069E0008200D358002B01D0FFF762FF1721A08847
:1069F000FFF768FDA08801F027FDA08801F0FEFDEB
:106A0000F7BDC046F95EFF1FF85EFF1F005FFF1F66
:106A1000F0B587B01D000CAB1B88070001930DABD0
:106A20001B88142002930EAB1B88160003930FAB38
:106A30001B880091049310AB1B88059304F044FF5E
:106A4000041E1AD0D0230370CB3B47708370C670EE
:106A5000062229000430002D11D004F095FF019B7F
:106A600021006381029B0098A381039BE381049B27
:106A70002382059BA37405F087F807B0F0BD04F0EE
:106A8000C3FFECE7F7B5009308AB1B8807000C20A9
:106A90000D001600019304F017FF041E13D0280008
:106AA00001F042FF00280FD00078D0232370C93BAB
:106AB000A370009B21002381019B6770A580E68065
:106AC000638105F061F8F7BD014B1878EDE7C0462A
:106AD000983DFF1F13B5040064890389C28881882B
:106AE000C0780094FFF7CEFF13BD000010B5044C32
:106AF0002068002803D004F027FE0023236010BD87
:106B0000045FFF1FA122F0B5818892004A43384BF1
:106B1000384F1B6804009B189D2292009B188279B5
:106B200089B01A603B68002B5FD01D78324B1B6820
:106B3000002B04D05B68002B01D000209847260072
:106B400008363100E079FFF7B7FD237DE0710200E0
:106B5000E0780493638A29000393238A0293E389EC
:106B60000193A38800933300FFF752FFE378002BD3
:106B70000BD1E289A379A18802920196E2792800DB
:106B80000092012201F0DAFEE0703B68002B20D079
:106B9000FFF7ACFF194D287800281AD0184B197848
:106BA000FFF778FE002814D02B78E67808200793AA
:106BB000A78804F089FE011E09D0D0230370CA3BC8
:106BC0004670837087808671079804F0DDFF00238C
:106BD0002B701721A088FFF775FCA08801F034FC0A
:106BE000A08801F00BFD09B0F0BD064B9DE7C04643
:106BF0003409FF1F045FFF1F185FFF1FF95EFF1FAF
:106C0000F85EFF1F983DFF1FF8B5070008000E0053
:106C100001F08AFE041E18D02620FFF78DFC051E09
:106C200000D12578062004F04FFE041E0DD000216F
:106C3000062204F0E9FED0232370C23B21006770D6
:106C4000A370A680E8B204F09FFFF8BDF0B585B050
:106C500001930AAB1B78070002930BAB1B7808006B
:106C60000D000092039301F05FFE061E22D010205B
:106C700004F02AFE041E1DD01022002104F0C4FEE0
:106C80002620FFF759FC002800D13078D02323704C
:106C9000C13BA370009B21002372019B677063724C
:106CA000029BA580A372039BC0B2E3720C9BE360BE
:106CB00004F06AFF05B0F0BDF7B50D00019001F0DA
:106CC00033FE071E20D00E2004F0FEFD041E1BD054
:106CD0002620FFF731FC061E00D13E78D02323800A
:106CE000C53B0622A370F91DE01C04F04DFE019B7C
:106CF0002A0063810123DD401A401D4021002273D8
:106D00006573F0B204F040FFF7BD0000F0B585B048
:106D1000029010000D0017000A9E039301F004FE7C
:106D2000041E31D0029B002B2ED1039B02795B07FE
:106D300024D5122313430422002E08D10B990029D5
:106D400005D10C99002902D10D9900291AD01A43B6
:106D50000D9B2271002B00D0C9E0002E00D1CFE0A6
:106D6000002D00D0CCE0606A002801D004F0ECFCDB
:106D70001C21300004F0C8FE606205E002239A4343
:106D80000E33D7E793432371654BBA00D458002CD8
:106D900000D1AAE0002E10D0236A002B03D11C20C2
:106DA00004F052FE20625E4BBA00D358186A0028E5
:106DB00003D01C22310004F0E7FD0C9B002B12D005
:106DC000574CBB001D596B6A002B03D1162004F0F1
:106DD0003BFE6862BB00E358586A002803D01622C5
:106DE0000C9904F0D1FD0D9B002B11D04C4DBC0033
:106DF0006659B36A002B03D1142004F025FEB0625B
:106E00002B59986A002803D014220D9904F0BCFD78
:106E1000380001F089FD051E67D0414BBA00D358F8
:106E2000002B62D01A6A3420002A00D11C389A6ADA
:106E3000002A01D0143080B20B9A002A01D01C30F5
:106E400080B25B6A002B01D0163080B204F03CFDAA
:106E5000041E4AD01822002104F0D6FD2620FFF798
:106E60006BFB0190002801D12B780193D023237074
:106E7000029B200063700A23294EA370039BBD0070
:106E8000A371AB59A780196A1830002905D01C22BC
:106E9000A06004F079FD200034307359996A00290C
:106EA00007D0030014221433E060029304F06CFD59
:106EB00002980B9B002B08D003001C221C330B995B
:106EC0002061029304F060FD02987359596A002909
:106ED00003D01622606104F057FD6B46210018793B
:106EE00004F052FE3800FFF7E3FC05B0F0BD1022BD
:106EF0000D9B0D991B69A018236204F045FD2CE73A
:106F00000B9B002B00D13FE7012D00D03CE7606ACE
:106F1000002801D004F018FC1C210B982AE7C04679
:106F2000005FFF1F10B5044C2068002803D004F058
:106F30000BFC0023236010BDF45EFF1F0B4B07B555
:106F40001A68002A01D100200EBD6946531C012099
:106F500012780731FFF772FC0028F4D00278012381
:106F6000100018401A42EED0EEE7C046105FFF1F37
:106F7000F0B51F4F01203B6887B0002B25D09B78D0
:106F8000059300F0B3FB002821D00A20FFF7D4FAC4
:106F900004000B20FFF7D0FA164B05001E78731E75
:106FA0009E413B68F6B2191DD878FFF757FB3B6846
:106FB0002900DA7A043303929A79019302920090BD
:106FC00033002000059A04F067FC07B0F0BDFFF71E
:106FD000B5FF002805D00620FFF7AEFA0400072011
:106FE000D8E70820FFF7A8FA04000920D2E7C04636
:106FF000F45EFF1FF05EFF1F70B50A4E0400337889
:107000000D00FF2B0DD0042004F05EFC011E08D003
:10701000D0230370CE3B45708370C470307804F089
:10702000B3FD70BDA83DFF1F70B5040006200D0024
:1070300004F04AFC011E0AD0D0230370CD3B8370BC
:10704000054B44701B688580187804F09DFD002C6A
:1070500001D0FFF767FF70BDF45EFF1FF8B5264F44
:1070600006003B680D001124002B05D10522234B9F
:107070001B78134202D112242000F8BD204A1024AC
:107080001268002AF8D01278002AF5D0DB0719D54B
:107090002B789A1E012A1AD80C2004F0D5FC132450
:1070A00038600028E8D000230A22437029000670C7
:1070B000023004F069FCFFF75BFF041E0AD0FFF703
:1070C00031FFD9E700F012FB0028E1D1E4E7002B03
:1070D000E2D0D0E70B4B1B78032BCDD11D20FFF75F
:1070E0002BFA094B18800028C6D0084B04211878C9
:1070F000074A04F0C1FABFE7F45EFF1FF15EFF1F0D
:10710000105FFF1FF05EFF1FEE5EFF1F1C5FFF1F83
:1071100060EA0000F7B50193194B14001A780523B3
:1071200006000F0012201A4221D0012920D1154B50
:107130001D68002D1BD002201F2C18D8002C02D057
:10714000019B002B13D0104B1F221E706E1C0021C0
:10715000300004F059FC01992200300004F014FCC6
:10716000310020002C70002F06D004F0B5FBFEBDCE
:10717000064B12201D68DCE704F04EFBF7E7C04623
:10718000F15EFF1F105FFF1FA83DFF1F0C5FFF1F79
:10719000F8B50F4E12243368002B17D01B780F3C24
:1071A000834213D100250B4F0221387804F06CFA8A
:1071B000094B042138781D8004F066FA074B28003B
:1071C0001D8033685C7004F057FB04002000F8BD9C
:1071D000F45EFF1F1C5FFF1F085FFF1FEE5EFF1FB7
:1071E00070B5012823D11B4C2388002B03D01A4AE9
:1071F0001578002D07D0194B1B68002B02D018788A
:10720000FFF7C6FF70BD3B2B02D93C3B2380F9E75B
:10721000134E0221307804F037FAFA2223889200C4
:1072200002215A43307804F077FB2580EAE70B4BC4
:107230001B68002BE6D00B4B1B785B07E2D5084B95
:107240000221187804F020FA0022024B1A80FFF77E
:1072500069FED7E7085FFF1FEC5EFF1FF45EFF1FAC
:107260001C5FFF1FF15EFF1FF8B51E4D2868002848
:1072700003D004F069FA00232B601B4E306800280D
:1072800003D004F061FA00233360184F05243B78E3
:1072900018002040234221D0154800F02BFA3B78FB
:1072A000234213D0202004F0CFFB2860002813D005
:1072B0002022002104F0A8FB202004F0C5FB041EBE
:1072C000306005D02022002104F09EFB002004E065
:1072D000286804F039FA2C601320F8BD00F00AFA8F
:1072E000F4E7C046105FFF1F0C5FFF1FF15EFF1F3A
:1072F0009C3DFF1F10B50A4C23681A1E0ED00028B3
:1073000008D10130587004F0B7FA002805D023687E
:10731000002B02D00021FFF787FE0122100010BDD4
:10732000F45EFF1FF7B5274E050033680191181E64
:1073300021D05C78244F012C30D1FFF7FFFD0028CD
:1073400025D02000FFF7F8F80400412814D91F4B7E
:10735000022118781E4A04F08FF91E4B3C3C1C8019
:10736000022233685A703B78002B14D1280001990F
:10737000FFF75AFE0120FEBDFA2292004243002A86
:10738000EED0124B0221187804F0C6FAE8E7FFF7B6
:10739000D3F80200F3E700233B70EBE73B78002BC8
:1073A000E8D1032004F090FA011E08D0D023037026
:1073B000CC3B457083703368187804F0E5FBFFF729
:1073C000B1FDD7E7F45EFF1FEC5EFF1F1C5FFF1FE0
:1073D00060EA0000085FFF1F10B5174983880200AC
:1073E0008B4220D011D815498B4217D01449002068
:1073F0005B1899B2012907D8926811785A42534113
:10740000D8B2FFF7F9FD012010BD0E4A00209B18ED
:1074100007229BB29A424041C0B2F5E783681878D0
:10742000FFF768FFF0E7836899785A7809021878BF
:107430001143FFF777FFE7E70A200000062000006E
:10744000F8DFFFFFAFDFFFFF014B18707047C0464A
:10745000A93DFF1F10B5064C207001F041FA2078BD
:1074600004F0B2F90521207800F062FD10BDC0469D
:107470001C5FFF1F0BB273B50D00002B00DBC4E0D7
:10748000884B187804F010FB041E0ED00378912B63
:107490000FD0A22B00D1A1E0834B1878FF2852D047
:1074A000210004F071FB00284DD1802000026840CB
:1074B00076BD43780F2B76D013D8052B70D00E2BCA
:1074C000EAD18088794B98422BD8794B98421BD8C7
:1074D000784B9842E0D1A3681878591CFFF774F8EC
:1074E00038E03E2BD8D18378032B74D06CD8012B95
:1074F0006ED0022BD0D1704B1B68002B23D05B6861
:10750000002B20D098471EE06C4BC0180C28C3D825
:1075100004F062F81DC2C2150BC20B0B0B3223C262
:107520003C00674BC0180728B6D8664B1B68002B79
:1075300009D01B68002B06D0200098470AE0A368FA
:107540001878FFF7C7F8200004F036FAADE7A06816
:10755000FFF762F800289FD0F5E7A3681B78002B9F
:10756000F1D0554B1B68002BEDD01B68002BEAD0E7
:10757000210055489847EDE74F4B1B68002BE2D0A0
:107580001B68002BDFD021005048F3E7504B1B68ED
:10759000002BD8D05B68002BD5D021004348E9E709
:1075A000FFF7EAF9CFE780884A4B984203D04A4B6D
:1075B000984200D070E7464B1B68002BC3D05B6835
:1075C000002BC0D02100D5E7153B012BBBD963E7C9
:1075D000FFF798FAB7E7FFF77DFAB4E73F4B1B7860
:1075E000042B07D100236A4613800179408800F0FC
:1075F000C5FCA8E7364B1B68002BA4D05B68002BAA
:10760000A1D00100364898479DE7012421420AD0C5
:10761000294B1B68002B04D05B68002B01D0002095
:107620009847012043E78B070AD5264B1B68002BA0
:1076300004D05B68002B01D020009847022036E779
:107640000421280008400D4200D131E7254E33883F
:10765000002B21D0013B9BB23380002B1AD1FFF7C6
:10766000DBF800280AD0204B1C70164B1B68002B3F
:1076700004D05B68002B01D020009847FFF7C6F8C4
:10768000694601F001FD6846FEF7FEFF1D20FEF78A
:1076900053FF308004200AE7024B187803F0F4FF10
:1076A000F8E7C0461C5FFF1FA93DFF1F0E2000002A
:1076B0000120000009100000145FFF1FFEDFFFFF24
:1076C000AFDFFFFF185FFF1F0C2000000B20000042
:1076D000FC5EFF1F0D20000013200000F15EFF1F65
:1076E000FFFF0000EE5EFF1FEC5EFF1F10B501F014
:1076F0009BF910BD014B18607047C046185FFF1F13
:107700000B880020162B01D817230420014A138070
:107710007047C046C65EFF1F00207047074A03003F
:107720001188814207D091880020994202D101300E
:107730008000101870470020FAE7C046245FFF1F42
:10774000F0B58F7806000D00C5B01E2F15D1FFF7DC
:10775000E5FF051E03D10024200045B0F0BD002246
:107760003B003100C078009200F0B2FB0400A81C7E
:1077700000F0D2FBFF23EB70EEE7264B06240393C9
:107780001B78FF2BE8D0182FE6D87B08224A013B54
:10779000DB0002929A589446002ADDD0029AD31850
:1077A0005B68002BD8D00878002802D14B78012BD9
:1077B00002D10624122FCFD107AFAB88697800978A
:1077C0006446AA68A047041EC6D1AB78029A5B083B
:1077D000013BDB00D318390030005B689847041E7A
:1077E0000BD1AB78042BB6D0039A3100107822006D
:1077F000009700F06DFB0400AEE76A78002AABD179
:10780000AA7805A93B88087130000A704B80FEF702
:1078100047FBA0E7AC3DFF1F70BD00111D4B37B506
:10782000050098420BD000290AD1FFF777FF002806
:1078300005D11948FFF772FF002800D0058037BD39
:1078400001291AD1FFF76AFF041EF8D001235B4219
:107850000380A378FF2BF2D0FE2B07D00023E07823
:107860001422009329001E3300F032FBA01C00F00C
:1078700053FB01235B426380E1E70229DFD1013939
:1078800001F0BEF80028DAD12800FFF747FF041EF8
:10789000DFD1D4E7FEFF0000FFFF0000022210B599
:1078A000074B52421A80074801325A809A80DA8088
:1078B00000F07EFA044801F025F8002010BDC04613
:1078C000245FFF1F417700111D7800110388F7B571
:1078D0000400002B02D102252800FEBD42680221CF
:1078E000137825485268FEF7A5FD00282ED0234FB7
:1078F00001253A88002AEFD0802321885B020125E8
:107900009B1A9942E8DC0C2004F09EF8061E31D048
:107910003B8822889C4600231800019561469DB251
:10792000491989B2AA421BD8002801D062443A8082
:1079300000233000082208C0210004F025F8104A76
:107940001368002B13D100251660C5E76268022179
:1079500013780C485268FEF76DFD0028C7D1BAE7CE
:1079600060681D014019418101330198D6E71A0072
:107970001B68E6E71325AFE7DEBD0011AA3DFF1F38
:10798000205FFF1FDCBD0011014B18707047C0461F
:10799000AC3DFF1F14230A0010B51A40194204D051
:1079A0000122102101F048F810BD4B06F9D4012046
:1079B00088434000F8E710B514008B0604D5012277
:1079C000102101F039F810BD08230A001A401942AD
:1079D00002D14BB2002B0FDA102101F02DF8002854
:1079E00008D02300F2331B78002BECD0F13423783D
:1079F000012BE8D10020E6E703208907FAD4E2E76B
:107A0000F0B51F00184B85B01C68019002910392DD
:107A1000002C27D1200005B0F0BDA5683301ED187A
:107A20006B89019A934211D3029A93420ED8002F88
:107A300004D10A9B002B10D12C00EBE73B002978E6
:107A4000039A6868FEF7F6FC0028F2D10136B6B258
:107A5000A388B342E1D82468DAE7A3680A9A5B896D
:107A60001380E9E70026F3E7205FFF1F37B50C001E
:107A70000A8849880123914217D3002A15D0651D31
:107A800023792A0002210A48FEF7D4FC102300289B
:107A90000BD023796188208800242A000094FFF706
:107AA000AFFF0A23A04200D0230018003EBDC0460D
:107AB000DEBD001113B50A000888498801238842F9
:107AC0000BD8002809D00024137905320094FFF761
:107AD00097FF0A23A04200D02300180016BD13B55B
:107AE0000A0008884988012388420BD8002809D059
:107AF0000024137905320094FFF782FF0A23A04285
:107B000000D02300180016BDF0B58BB003904A8852
:107B100008880E000123824255D3002853D0002349
:107B2000012704AC23700022718813000092FFF734
:107B300067FF051E3ED02078002835D12B78022B18
:107B400018D167706A8983000130E31880005A8079
:107B500069680222201803F017FF23780133DBB293
:107B60002370042B19D93B006889013080B2002BA7
:107B7000D9D01FE002236370122358436A89231867
:107B800004305A8069681022201803F0FDFE237823
:107B90000133DBB22370002BE5D10C4A6B899B18B3
:107BA0005A425341DBB2DFE76378012BE4D12B78F3
:107BB000022BC7D022780A23002A04D02100039880
:107BC000FEF798F9002318000BB0F0BD0100FFFF8D
:107BD0000F4BF0B504001868002816D083685D8943
:107BE000A54207D88288AE18B44203DA12019A1867
:107BF000934201D10068EFE71E005F891036A7426B
:107C000004D1002900D00D801800F0BD3300EFE74B
:107C1000205FFF1F70B505000C0008880021FFF7EA
:107C2000D7FF03000120002B04D022002800197A7E
:107C3000FFF7C1FE70BDF7B50C00002501902300D1
:107C4000EE331B78AB4201D800200AE06B00E65A05
:107C500000213000E718FFF7BBFF002802D1268083
:107C60000130FEBD017A0198FFF794FE002802D092
:107C70003B882380F5E70135EDB2E0E710B504005D
:107C800008880021FFF7A4FF03000120002B03D088
:107C90002000197AFFF77EFE10BD0000054B1B681F
:107CA000002B01D1180004E09A6852898242F6D173
:107CB00098887047205FFF1FF0B50E27002687B019
:107CC000039302ABFF183E8005001F4B4089140050
:107CD000984207D02B78013000976A6880B2FFF78E
:107CE0008FFE060002212B7818486A68FEF7A2FB77
:107CF00000280FD06C892000FFF7D0FF002802D0A9
:107D0000013C0419A4B2039B002B00D01C8030005E
:107D100007B0F0BD02212B780D486A68FEF78AFB98
:107D20000028E7D102212B780A486A68FEF782FB17
:107D3000002807D0002EDED03B88A342DBD1748917
:107D4000013CDFE76C89DEE7FFFF0000DEBD0011CC
:107D5000DCBD0011DABD001110B50C00FFF7DEFC30
:107D600003000220002B0AD0002C00D023609B7857
:107D70001720FE2B03D00138FF2B00D1002010BDAF
:107D800073B50D0001A904001600FFF7E5FF1728E1
:107D900005D0002E04D129002000FEF727F976BD7A
:107DA00001221021200000F047FE0028F3D0F6E762
:107DB000014B18607047C046305FFF1F37B56B46F8
:107DC0009D1D010004000222280003F07DFE2B8887
:107DD000B02B0ED12379122B09D12300FA331B7853
:107DE000012B06D10121608800F0E0F801E01B2B97
:107DF000F8D037BD10B5054B0421187000F098F885
:107E0000FFF74CFDFEF770FB10BDC046345FFF1F4F
:107E10000020F0B50BB20F0087B0834234DA274B55
:107E2000187803F041FE051E2BD00378A02B25D136
:107E300003AE3100FEF7E4F8041E0BD1B378DB0784
:107E400024D51F4B06341B68002B03D031006888F3
:107E500098470400A868002801D003F08DFC002C8E
:107E600008D1184A039B1340174A934206D0B378AF
:107E70001B2B03D00121688800F098F8280003F03C
:107E80009BFD80200002784007B0F0BD0F4B1B68BF
:107E9000002B10D0310068889847041EDAD0737820
:107EA000002BD7D1B27801A90A704B800C71688879
:107EB000FDF7F6FFCEE70624F1E7C046345FFF1F6B
:107EC0002C5FFF1F00FFFF0000011200305FFF1F4B
:107ED000F7B50190FC200D0017001E0003F0F4FC24
:107EE00004001320002C12D0B02320002370089B24
:107EF000F4226770658026710830002B08D01900C5
:107F000003F042FD2100019803F03EFE0020FEBD7B
:107F1000089903F079FDF5E710B5041E06D0007846
:107F2000FD2803D803F000FCFF23237010BD0000E0
:107F30000A1F93B210B504000220032B05D882401B
:107F40000020024BD1529B189C7010BD545FFF1F44
:107F50000B8870B5043B04000D000220032B0BD8E6
:107F60000121200000F04CFD03001420002B03D061
:107F70002900200000F0DEFB70BD000007B51300F3
:107F8000034A00920A00012100F02CFC0EBDC046FD
:107F9000B981001107B5019203220092024B0A0039
:107FA000122100F049FC0EBD3782001107B56B4667
:107FB00001AA11800449D88008780633012802D12B
:107FC000190003F049FD07BD355FFF1F0C4B10B5CD
:107FD00018700023FF210B4A138013819381938033
:107FE000094A53801370517293819372D174D38272
:107FF0001375517703F0F8FC00F0FCF910BDC04692
:10800000645FFF1F545FFF1F365FFF1FF0B58DB029
:108010006B46002003910C229B5E834200DBB0E0A4
:108020005D4B187803F040FD051E00D1A4E00378F5
:10803000902B00D09DE006AF01004688380000F08C
:1080400013FA79680400002900D19CE03B88052BD5
:108050006ED13B89032B1CD905AC200000F0A2F89F
:108060006288172A61D83989131D994231D17968FC
:10807000237804310291D90738D5607800F08EF961
:10808000071E06D0002303712378012B08D0132B81
:1080900023D0A868002800D178E003F06DFB75E0DC
:1080A0006288029909A800F0A6F80290380000F052
:1080B0008BF909AA2378387A0192002231000092C4
:1080C000029A00F012F9380000F064F9029B002BCC
:1080D000DFD0300000F080F9DBE70378032BD8D144
:1080E0006288029909A800F0D6F8DEE7122B13D1B6
:1080F000029909A800F0B5F8021EEAD127498B8839
:10810000002BC6D0887909A9237801916178009164
:10811000310000F0EAF8BCE7002302AA93833000A4
:10812000617809AAFFF72AFFB3E71D4B0993F6E729
:10813000042B02D09A1F012AABD8184A043B9B009B
:10814000995A0029A5D0D218907831003A0000F051
:10815000AEF800289DD13B88042B03D001213000CC
:10816000FFF724FF012C04D1A868002801D003F0F8
:1081700003FB280003F020FC8020039B0002434007
:1081800018000DB0F0BD012800D182E701213000B8
:10819000FFF70CFFEDE7C046645FFF1F545FFF1F52
:1081A000010017000B7803704B784370CB788A7806
:1081B0001B021343438070470A88030002700A8839
:1081C000120A42700A88012A06D14A8882704A88B7
:1081D000120AC2700420704702208242FBD14A88F2
:1081E00004309A704A88120ADA708A881A718A886A
:1081F000120A5A71EFE710B50400012082420CD92F
:108200004B780A781B0213432380834206D1CB7834
:108210008A781B0213436380002010BD022BFBD120
:10822000CB788A781B02134363804B790A791B024F
:108230001343A380F0E70B8803700B881B0A43707D
:108240004B8883704B881B0AC3708B8803718B88A3
:108250001B0A4371CB888371CB881B0AC37108202A
:10826000704703000120082A14D14A7808781202C6
:1082700002431A80CA788878120202435A804A79E7
:108280000879120202439A80CA798879120202435D
:108290000020DA80704710B504000120022A05D1C1
:1082A00000204B780A781B021343238010BDF8B5D9
:1082B000060010200F00150003F006FB040001204B
:1082C000002C0ED0A0230C22290023806780201DC3
:1082D000002D07D003F058FB2100300003F054FCC0
:1082E0000020F8BD03F090FBF6E7F7B51E00009004
:1082F00008AB142017001D78019103F0E5FA041E65
:1083000012D0A2230370019B47704380099B057123
:1083100046710C220830002B07D0190003F034FB03
:108320002100009803F030FCF7BD099903F06CFBC5
:10833000F6E737B5041E0FD04388002B0CD000257C
:10834000C1881323007A172201950095FFF7CDFF0E
:10835000FF2365806372257037BD000010B50C499E
:1083600004004A88002A09D08B89002B05D0002000
:10837000CB8A0222834201D010BD012213000A20C1
:10838000434300204032C854C81842800472F3E7C7
:10839000365FFF1F0023438003707047094B0021A5
:1083A0001A0010B55C88002C06D01C79844203D1D9
:1083B0000A234B43D01810BD01310A330329F1D1F0
:1083C0000020F8E7365FFF1F10B50400407A03F085
:1083D000ABF9FF23637210BD7047043010B580B253
:1083E00003F0EAF9002803D00421494203F07CFBA2
:1083F00010BD000070B50025104CA0682580A58137
:10840000A580A84202D003F0B7F9A56000250C4C66
:108410000C4B606D1D80230058331D70A84202D0A4
:1084200003F0AAF9656500256068002801D003F013
:10843000A3F9013508340A2DF6D170BDFC5FFF1F8A
:10844000A05FFF1FF05FFF1F70B5041E09D1054D2F
:108450002880A881A880A868002802D003F08CF9A1
:10846000AC6070BDFC5FFF1FF0B54B8885B0019319
:10847000002343600A7905000F00022A00D07BE048
:10848000CA88032A17D98B685E7819783602DC7897
:10849000D8790E4399781B7A24021B020C430343BC
:1084A00053495BBA0B80331D93421ED1042C04D078
:1084B000631F022B0ED9012015E0019A4D4B1201CA
:1084C000D35A002B06D00198FFF7BEFF4A4A136922
:1084D000013313610421B8682E812C80494203F0D6
:1084E00003FB6860002005B0F0BD434D042C06D0AE
:1084F000631F022B0FD9EB680133EB60DBE7019AB6
:108500003C4B1201D35A002B05D00198FFF79CFF7A
:108510002B6901332B61374B30000293019B029A88
:108520001B010193002301998C468B521300634475
:108530009C8003939E81FFF750FF039B041E98606D
:1085400016D00421B868494203F0CEFAFA88010037
:10855000043A200003F018FA0199029AFB888A5A1B
:10856000043B9B18029A8B522B6801332B60A2E7C5
:10857000AB690133AB619EE71E4B0293019B1E0169
:10858000029BF35A002B2DD002998C19A068002869
:1085900028D0012A26D1FA889B189BB27352A18950
:1085A000994217D39B1AC018B96803F0EDF9029BE2
:1085B000A289F35A934200D07DE700222B81A38841
:1085C0002B80A3686B60029BF2520B4A5368013305
:1085D000536070E7084A9368013393600198FFF78E
:1085E00033FF68E7044A536901335361F6E7C04635
:1085F000665FFF1FFC5FFF1F6C5FFF1F70B5051EEE
:1086000015D10B4C0B4B1880230058331870606D3C
:10861000002802D003F0B0F8656525005035606889
:10862000002801D003F0A8F80834AC42F7D170BD9F
:10863000A05FFF1FF05FFF1FF0B51700A12285B0FC
:10864000920001934243394B06001B680C009B18B3
:10865000D933FF331D78FDF741FF0430854204DD37
:108660003000FDF73BFF0430C5B2BD4207D33A00EE
:1086700000213000019B03F01FF805B0F0BD290078
:10868000380003F001FA2300C6B250331E70039382
:10869000019B29006365380003F0D6F8CBB2029342
:1086A000002B02D0039B01361E700026230050339E
:1086B00003931B78B34204D8606D002831D10020A9
:1086C000DBE7029A2800002A04D0013B1000B342E5
:1086D00000D02800F700E719387002F075FF7860C5
:1086E00000280ED03A78019903F04EF9019A3B78B0
:1086F0000136D3180E4A0193D369F6B20133D36120
:10870000D4E7039B18706065A74205D1084A13207F
:10871000D36A0133D362B0E7606803F02DF8083400
:10872000F2E703F029F800236365C8E73409FF1F67
:108730006C5FFF1FF7B50D0007000421686803F0A8
:10874000D3F92B89040003702B891B0A43702B88F3
:1087500083702B881B0AC3702E8902250436F6B25B
:10876000F42E15D81B4B9F4214D10C2003F0ACF80B
:108770001135011E0CD0902303708E3B0371043B16
:108780004380154B8460C680187803F0FDF90025FE
:108790002800FEBD5C237B43104AD3180093583356
:1087A00001931B78002B0FD1030032003800009991
:1087B000FFF742FF019B05001B78002BE8D1380032
:1087C000009902F0C9FFE3E7054A0725536A013320
:1087D0005362DDE7FEFF0000645FFF1FA05FFF1F25
:1087E0006C5FFF1FF0B587B0009017200F001600D8
:1087F0000193FFF7F2FD1325041E19D00C98031EF8
:1088000002D00199201D9847030AE370052302AAAC
:10881000A0700430908127700098667003A993803F
:108820000494FFF787FF051E02D0200002F0A4FF8A
:10883000280007B0F0BD0000F0B587B01F000CABFA
:108840001B780391059301210DAB06001C7804925F
:1088500000F0D6F81425002821D02000FFF77EFD77
:108860000135041E1BD01149059B0A7803700132A3
:10887000D2B2131EC68001D101231A000B702271DF
:108880003000049B03990097FFF7ACFF051E09D148
:10889000230021000648074A093303F0ADF82800F9
:1088A00007B0F0BD002363802370F8E7685FFF1F07
:1088B0003383001130750000F8B505000E00064C3A
:1088C000064F2368002B02D031002800984704345B
:1088D000BC42F6D1F8BDC0460C60FF1F2060FF1FF0
:1088E0000123064A5B425380002313715362044AFA
:1088F000136053609360D360136170472060FF1F63
:108900000C60FF1F0200002310B506499C000859A7
:10891000002801D1625010BD0133052BF6D1132080
:10892000F9E7C0460C60FF1F034A5388181A4342F8
:1089300058414042104070472060FF1FF0B585B09D
:1089400002930AAB1F780CAB1B88009008000E0046
:1089500001920393FFF7E8FF05001120002D1BD1C2
:108960000E48FFF7E1FF04001520002C14D006226A
:108970000B99A771E01D03F007F8019B30002371EC
:10898000029B29006371009B66802370039B6562D4
:10899000E381FFF791FF280005B0F0BDFFFF000065
:1089A00010B5FFF7C1FF04000220002C12D0608830
:1089B0000121FFF781FF606A002801D002F0C4FEA8
:1089C00028220021200003F01FF8012300205B4231
:1089D0006380207110BD000030B5074A074C5588F0
:1089E000010013780020A54204D05B1A59424B4184
:1089F0005842104030BDC0462060FF1FFFFF0000FE
:108A0000084A10B501230C00904208D0FFF78CFFF4
:108A1000031E04D0037923405A1E9341DBB2180091
:108A200010BDC046FEFF0000024B1879431E98415E
:108A3000C0B270472060FF1F70B504000D00160023
:108A4000FFF772FF002804D10D4B9C4200D0143078
:108A500070BD416A03790520002907D012221A400F
:108A6000102A02D10520002EF2D10F20DB06EFD50F
:108A7000897E0C20A9428941494249420840E7E7E2
:108A8000FEFF0000030010B5002800D110BD034810
:108A9000034A41889142F9D09847F7E72060FF1FC9
:108AA000FFFF0000002330B5C45CCD5C6C40D454A3
:108AB0000133102BF8D130BD0F23002210B5C45C58
:108AC00064002243CA54C25CD209013BF7D210BDF4
:108AD0000200010010B52032103102F07DFF10BD00
:108AE000F0B58BB00390102005931700049102F0AD
:108AF000ABFF0090102002F0A7FF009B1324019011
:108B0000002B05D000280CD11324009802F01CFE85
:108B1000019B002B02D0180002F016FE20000BB0C3
:108B2000F0BD102002F090FF0600102002F08CFF34
:108B300013240500002E00D1AEE0002819D0102229
:108B4000002102F061FF32002900039802F044FF87
:108B5000041E0ED133787F2B51D830000099FFF7D7
:108B6000ABFF009B1B787F2B53D801990098FFF730
:108B7000A3FF300002F0E8FD002D02D0280002F033
:108B8000E3FD002CC1D1102002F05EFF0600102092
:108B900002F05AFF0290002E7CD0002878D03A00D4
:108BA0000F3223000125121105D00F333B4015B2BF
:108BB0005A4253411BB26A1E1201002B33D0049B50
:108BC000D2B298180099029AFFF76CFF013D10226B
:108BD0000021300002F018FFADB2049F2D017D1975
:108BE000AF4242D0002C33D0300002F0ADFD029BEA
:108BF000002B00D189E7180002F0A6FD85E72900C7
:108C00003000FFF759FF28002549009AFFF74AFF77
:108C1000A7E729000098FFF74FFF28002049019A95
:108C2000FFF740FFA5E70F210F4004998A18D9B23A
:108C30008F4208D9D15C06A819540133102BF6D104
:108C4000029A0199C0E7791A48424141C901F2E705
:108C50003900300006AAFFF725FF3200039806A965
:108C600002F0BAFE10370400BAE7002CBCD1300085
:108C7000029906AAFFF716FF320006A9039802F030
:108C8000ABFE082204003100059802F07DFEABE740
:108C90001324A9E71324AAE7002800D06EE733E7DE
:108CA000E4BD0011F0B58BB00F0016000225009056
:108CB00000283FD0002A3DD00B1DDBB218000293E4
:108CC00002F0C2FE1135041E34D0FDF747FD050049
:108CD0003A000099201D02F03FFFEBB20393E370CE
:108CE0002B0CDBB22F0A00936370FFB22B0E2370A4
:108CF000A7700193FDF72CFD1022010006A802F0D9
:108D00002BFF2100029A04AB06A8FFF7E9FE051E1F
:108D10000DD1039B08223370009B04A9B370019B03
:108D20007770F370301D02F017FFFDF71DFD200076
:108D300002F00AFD28000BB0F0BDF0B58FB00D00B9
:108D4000149E039004920593002A03D1022420006C
:108D50000FB0F0BD002EF9D00398FFF7E5FD142405
:108D6000071EF4D07278337812021A43B3781B04CA
:108D70001343F27812061A43036A0192934201D315
:108D80000133E3D1002D03D03B7901249B07DED5CD
:108D90000822002106A802F037FE059B13240433A5
:108DA000DBB21800029302F04FFE051ECFD0059AE9
:108DB0000499043002F0D0FE04223100280002F0B1
:108DC000CBFE3900102210310AA802F0C5FE29009E
:108DD000029A06AB0AA8FFF783FE041E0FD10822F1
:108DE00006A908A802F0B8FE0822311D08A802F062
:108DF0005BFC012807D101990398FDF7C9FC280005
:108E000002F0A2FCA3E70124F9E7000070B51C4CB6
:108E100005002368181E10D0002D14D11A78002ADE
:108E20000CD1981C083202F0AFFD02F015FC0135A0
:108E3000002808D123681D70012070BD0A33180076
:108E4000082202F0A1FD2368002BF5D0122002F0C9
:108E50003BFD061E0DD0C123216803704570023111
:108E60001022023002F090FD23683100587802F0A1
:108E70008BFE206802F068FC00232360DCE7C0461C
:108E80004860FF1FF8B504002020FDF755FB0D4E8C
:108E9000A700BB590500002B0DD000280BD0D878B7
:108EA000FF2809D108492A000C55F3590748033314
:108EB000611802F0A1FDF8BD290002F03DFE002876
:108EC000F0D1F8E76460FF1F4C60FF1FDDA00011C8
:108ED00070B5064D84006359002B05D0D87802F098
:108EE00023FCFF226359DA7070BDC0466460FF1F27
:108EF00070B506008CB00C001500002130226846C9
:108F000002F082FD31001022684602F025FE1D208D
:108F100021000322684402F01FFE6846FFF7D8FDD7
:108F20002D21040003222800694402F015FE2000D0
:108F30000CB070BDF0B50700160097B001931CABE4
:108F40001D7830221EAB00910AA800211C7802F087
:108F50005BFD102239000AA802F0FEFD102200215C
:108F600002A802F051FD0722310002A802F0F4FD30
:108F7000072202AB9818631E9C41019902F0ECFD98
:108F800002AB9C732B005A1E934102AAD37300219B
:108F9000102206A802F038FD06221D9907A802F04B
:108FA000DBFD1A2002ABC01806221F9902F0D4FD87
:108FB000102200990EA802F0CFFD102202AB0EA9DC
:108FC00008781C78013A6040D2B208700133013150
:108FD000002AF5D10AA8FFF77BFD102212A9040090
:108FE0000EA802F0D1FC102206AB0EA908781D785D
:108FF000013A6840D2B2087001330131002AF5D13C
:109000000AA8FFF765FD044310222098E4B212A9D4
:1090100002F0A2FD200017B0F0BD70B50E001400E4
:109020008CB00100102268461D0002F095FD310051
:10903000082204A802F090FD2100082206A802F0F0
:109040008BFD6846FFF744FD04001022280008A9A4
:1090500002F082FD20000CB070BDF8B506000D00D6
:1090600000243719AC4200D3F8BD02F025FC030AF6
:109070003B70631CDBB201379D4203D90234F054CC
:10908000E4B2EEE71C00EDE773B506000C00022524
:10909000002819D0002917D0032101A8FFF7DDFF10
:1090A0006B469A793F231A40013313436A463000D6
:1090B000937101A92200FFF71BFF051E04D10322B3
:1090C000E01C01A902F060FC280076BD0378580777
:1090D000DA08C00FD20080009B0710439B0F184393
:1090E000C0B2704707230B40C908C9000B43037087
:1090F0007047000070B50400FFF7EAFE134DA400AE
:109100006359002B21D0186A002801D002F01CFB03
:109110002B59986E002801D002F016FB2B59D86EFF
:10912000002801D002F010FB2B59186F002801D045
:1091300002F00AFB2B59586F002801D002F004FB03
:10914000285902F001FB00232B5170BD6460FF1F02
:109150000E4B8000C35870B50C00002B0FD09D68DB
:10916000002D0CD02B78201D0B706B784B70A97CD8
:10917000FFF7B8FF2B7E23726B69E36070BD10228E
:109180000021200002F040FCF8E7C0466460FF1FA9
:10919000014B18607047C0466060FF1F074A03001C
:1091A0008000825810B5002A06D0D088984203D19A
:1091B000012901D1FFF79EFF10BDC0466460FF1F6B
:1091C000F0B5264E95B087000B93BB590500099169
:1091D00012200A92002B31D0D888FFF7A5FB04009B
:1091E0001420002C2AD0280010A9FFF7B1FFBB598A
:1091F0001E781D6A002E23D00895FDF7EFFA0700B0
:109200000020FDF7F1FA0790A379E61D069310AD53
:109210000CA9089800F0E2FA0EA9280000F0D7FA8D
:109220000B9B0A990493069B09980293079B03964C
:10923000019300970EAB0CAAFFF77CFE15B0F0BDB2
:10924000FDF7CCFA06903000FDF7CEFAE31DA779C2
:10925000079310AB06000893DAE7C0466460FF1F6F
:1092600030B50C4C85002A59030085B00120002A36
:109270000ED018006946FFF76BFF2B591A78D88873
:10928000054B002A00D1054B6A46072100F0D9FBA7
:1092900005B030BD6460FF1FCF970011DD9700114E
:1092A00030B5094C8500295985B010226846253112
:1092B00002F06AFB2A591121044BD0886A4600F05B
:1092C000C0FB05B030BDC0466460FF1F7998001137
:1092D00030B5094C8500295985B0102268463531D2
:1092E00002F052FB2A591121044BD0886A4600F043
:1092F000A8FB05B030BDC0466460FF1FB7980011E1
:10930000F7B54D4F86001020F4590D0002F09CFB7C
:10931000F3592062186A132200286CD0033A2900FE
:109320009C6802F031FBF3591A780192002A58D157
:109330001E6A227D317B944651400122019F1142D9
:1093400001D167461740217D914339432175377B11
:109350004F40BC4660460027800701D44F081740A5
:10936000012102208F40227D82433A432275377BC0
:109370005740BC4660460027400701D497080F407D
:109380000420227DBF0082433A432275627D00277C
:1093900094466046727B42400A4201D167460F40C4
:1093A0000121627D8A433A436275777B5740BC4610
:1093B00060460027800701D457080F400220627DD5
:1093C0007F00824317436775767B00227E407607D5
:1093D00001D4BA080A400426617D9200B1430A43D1
:1093E00062756A78002A08D06278002A05D00522C2
:1093F0000533DA7700221000FEBD042229791142DC
:1094000005D1A17C114202D10533033AF1E7019A5B
:1094100021782C78002A02D10A0021001400182299
:109420000429E8D8042CE6D805206043034A053314
:109430001218525CDDE7C0466460FF1FF4BD0011E6
:1094400010B50A001121024B00F0FBFA10BDC04616
:10945000139900110B0030B587B001AD2B806B461E
:1094600004001100981D082202F08EFA2A000B2138
:109470002000024B00F0E5FA07B030BD3B99001127
:1094800010B50A001121024B00F0DBFA10BDC046F6
:109490008F99001113B50B0011006A4613706B46CB
:1094A00004000622581C02F06FFA6A4608212000C8
:1094B000014B00F0C6FA13BDAF99001110B50A00B8
:1094C0001121024B00F0BDFA10BDC046FF990011FA
:1094D0007FB505000B4BAA00D4580800002C0FD014
:1094E000666F237FE28821780396266F0296E66EE8
:1094F0000196A46E0094FDF709FC2800FFF7FAFD21
:109500007FBDC0466460FF1F10B51721FFF7E0FF65
:1095100010BD000070B50A000D00064B02210400CA
:1095200000F08FFA060029782000FFF7D1FF300005
:1095300070BDC046DF98001170B586B000236A4642
:109540001370836804001D78681E0A2859D801A981
:1095500002F0DAF8060633373B3F43474B4F5300E0
:10956000180000F042F9062312284BD000281BD126
:109570006088FFF7D9F90823002813D04279002A20
:1095800047D1264B1A78072312070BD5244B1A68AC
:109590000723002A06D01668002E03D0290001AA4E
:1095A000B04703006A4613706B461B786088002B37
:1095B0002AD1FFF767FC06B070BD180000F06CF907
:1095C000D4E7180000F087F9D0E7180000F093F90D
:1095D000CCE7180000F0ADF9C8E7180000F0C3F9B7
:1095E000C4E7180000F0F6F9C0E7180000F0F6F93B
:1095F000BCE7180000F013FAB8E7180000F013FAFF
:10960000B4E707236A46137069466088FFF782FF54
:10961000D1E70523012AC5D1024BB8E7F15EFF1F50
:109620005C60FF1F6060FF1FF8B52C4F8600F35988
:1096300004000D00002B40D0DA8882423DD15A78D8
:10964000062A33D11A78002A2ED0012099681A6A86
:10965000097D014206D0157B054203D007225A70CE
:109660000120F8BD0220014204D0157B054201D043
:109670000922F4E70420014204D0127B024201D007
:109680000B22ECE7164B1B68002BE9D05B68002B24
:10969000E6D020009847BB5900215B78122BDFD120
:1096A0002000FFF715FFDBE70E4BECE7112A04D192
:1096B000002900D032252900F2E7002D08D1200032
:1096C000FFF732F9002803D0102302791343037106
:1096D00021002800FDF798FAC2E7C0466460FF1F2A
:1096E0005C60FF1F6060FF1F70B50E4E8500AB59B8
:1096F0000400002B13D01B78002B11D10A4B1B68E0
:10970000002B04D05B68002B01D0200098477359D0
:109710005B78122B03D100212000FFF7D9FE70BD2A
:10972000024BECE76460FF1F6060FF1F5C60FF1F7F
:10973000094B8000C3581020002B0CD01A6A002A55
:1097400009D09B68002B06D0127A1B7E101C9A420F
:1097500000D9181CC0B270476460FF1F70B50300C9
:109760000D0014000220002A30D000292ED01370E2
:109770000B78081D53704B789370FFF7A7FCE070CF
:10978000012002212B7A23716B7B034063716A7B7A
:109790000A401343042263716E7B164033436371A6
:1097A0006E7BF608F600334363712B7B0340A37195
:1097B000287B014000200B43A371297B0A401343FF
:1097C000A3712A7BD208D2001343A37170BD10B5D8
:1097D0000A0001000120FFF7C1FF10BD10B50A000B
:1097E00001000220FFF7BAFF10BD70B506000C00A3
:1097F0000220002E30D000292ED07378201D0B704F
:10980000B3784B70F178FFF76DFC01223579257242
:1098100071794B10080013409340104003438810A7
:1098200010408000C9080343C9000B436373B1793A
:109830004B1008001340934010400343881002402F
:109840009200C9081343C9000B4321202373FCF77E
:1098500073FE854201D2122070BD2220257AFCF7CA
:109860006BFE8542F7D823781820042BF4D8637850
:10987000012BF1D80020EFE7030010B502200029EA
:1098800009D0002B07D00322481C0A7019000D32A2
:1098900002F07AF8002010BD03000222080010B583
:1098A000002B06D0002904D00E32591C02F06CF8AF
:1098B0000022100010BD030010B50220002909D0BD
:1098C000002B07D00422481C0A7019000C3202F049
:1098D0005BF8002010BD10B5FFF7DEFF10BD0300E0
:1098E0000220002906D0002B04D0052200200A7097
:1098F0001B784B70704703000220002B08D0002912
:1099000006D05B7800200B70013B082B00D9183083
:109910007047030010B50220002909D0002B07D0A2
:109920000622481C0A7019000A3202F02DF80020A5
:1099300010BD10B5FFF7B0FF10BD02000B000220F4
:1099400010B500290ED0002A0CD0072119701188FB
:1099500059701188090A997011180822D81C02F050
:1099600013F8002010BD03000A00022010B5002BE0
:109970000CD000290AD09978587809020143118047
:10998000901CD91C082201F0FFFF002010BD03002D
:1099900010B50220002909D0002B07D00822481C4E
:1099A0000A701900921801F0EFFF002010BD0200AC
:1099B0000B00022010B500290BD0002A09D0092184
:1099C0001970117818185970511C062201F0DCFF2B
:1099D000002010BD10B5FFF75FFF10BD02000B00A7
:1099E000022010B5002A09D0002907D0517819703B
:1099F00011180622581C01F0C7FF002010BD0300FB
:109A000010B50220002909D0002B07D00A22481CDB
:109A10000A701900063201F0B7FF002010BD10B522
:109A2000FFF73AFF10BD02000B00022010B5002A1C
:109A300006D0002904D018005178FFF753FB00200E
:109A400010BDF0B585B017001E006A46062305005C
:109A5000080091819380FEF7C0FC1324011E029040
:109A60000CD03800B047041E05D1280001A9FEF72C
:109A70006FFA041E02D0029801F07EFE2800FFF764
:109A800001FA200005B0F0BDF0B504008BB00191E3
:109A900015000021102202A801F0B6FF334EA700E6
:109AA000B85900283CD0C388A34239D10378002B91
:109AB00036D14278062A18D10200010055323531DC
:109AC0000C3006ABFFF7A9FA002829D12000FFF7D8
:109AD0002FFE020006A902A801F056FF200002A9ED
:109AE00001F0AAFF01200BB0F0BD816E002917D054
:109AF0000B8A112A28D19D420ED101981231093AC0
:109B000001F0D2FD012807D1BB5920009D6EFFF75F
:109B10000FFE29000200DEE732212000FFF7D8FC0B
:109B20002000FEF701FF061E1BD0416A002918D055
:109B30000B8AAB4215D108220198123101F0B4FD15
:109B400001280ED1716A0AE09D42E9D108220198EC
:109B5000123101F0A9FD0128E2D1BB59996E8A7E2C
:109B6000B9E7200001F0A0FEBCE7C0466460FF1F1B
:109B7000F0B56B4D87007E5985B033780290039322
:109B8000002B00D087E0B368346A01937078062810
:109B900017D101221B7D134202D0217B114218D123
:109BA0000222134202D0217B114251D104221342DE
:109BB00003D0237B134200D08BE0019B5A7DEB59ED
:109BC00091E007380428F8D801F09EFD032E426783
:109BD0008300B36E002B03D11C2001F035FFB0666B
:109BE000EB599C6E002C1CD010220021200001F0AB
:109BF0000BFF0298FFF79CFD01002000FFF72DFAF4
:109C000001F05AFE2082200008211230FFF725FAC9
:109C10000298FFF78DFDA076EB592100D888FFF759
:109C20000FFC0822EB591CE0B36E002B05D01A0084
:109C3000198AF0881232FFF70DFC0222019B197D70
:109C4000EB5911423DD0207B10423AD0073208E058
:109C5000F488FCF7DBFD01002000FFF711FC0A226D
:109C6000EB595A70029B9C002A595378073B042BEE
:109C700011D8D088FEF758FE00284ED0C3895A0864
:109C8000D2182849029B0298CB542B59411804330F
:109C9000254801F0B1FE05B0F0BDFCF79FFD0300C3
:109CA0000120834201D100200393EB59DE88FCF7A9
:109CB0009BFD039902003000FFF7ECFB019AEB5982
:109CC000117D042211420CD0217B114209D00B22BC
:109CD000C7E7F688FCF73CFD01003000FFF7EEFB1C
:109CE0006BE7019A527D01210A4204D0607B084251
:109CF00001D00C22B5E702210A4204D0607B084261
:109D000001D00E22ADE704210A4204D0627B0A4250
:109D100001D01022A5E71222A3E7FA225200B0E7F1
:109D20006460FF1F6860FF1FE7A0001110B5064BBD
:109D30001A780423100018401A4200D00348FFF795
:109D400027FA002010BDC046F15EFF1FB03DFF1F87
:109D500070B50400FFF7D4FA051E43D12000FFF7C9
:109D60007FFA234EA400A0598268937CDB0708D5B4
:109D70000321036A1B790B40012B02D1017F0B43A6
:109D80000377431DD97F8B1E022B0DD8022900D0EB
:109D90000121C088FCF790FF042133591A7F5970C4
:109DA0000A431A77280070BD01290CD10223102222
:109DB000437000210C3001F027FE3059102135305E
:109DC000FFF74BF9EEE70529ECD10223D1184370D8
:109DD00010220C3001F0D8FD04233259117F0B43BF
:109DE0001377EAE708251828DCD1053DDAE7C046F5
:109DF0006460FF1FF0B58BB0059143887E4F9E00D5
:109E0000F45915000493002C15D1012902D000202B
:109E10000BB0F0BD101D57781678FFF757F9EB68B7
:109E2000320002932B7A0499019300903B002000AA
:109E3000FCF70CFFEBE7E388049A934201D008207B
:109E4000E6E72378012B00D1D4E0059B581E0928B2
:109E500000D9CFE001F058FC05CE0A29CC506C8522
:109E60009AB229000498FFF773FFD1E72000290078
:109E70001022453001F088FDB9594B78042B02D1EE
:109E8000013B4B70C3E70B000A00253335320C3120
:109E90000498FFF795F90498FFF702FA0522431E8C
:109EA0009841BB59C0005A70B2E720002900102227
:109EB000553001F069FD049B4F4C9D0029590498D1
:109EC0000A0006AB55320C31FFF77AF929591022F6
:109ED000453106A801F0E8FB012808D10498FFF7F6
:109EE000F7F90590002804D106222B595A700598DD
:109EF0008EE708230593FAE763780C2B7AD1E36E9B
:109F0000002B03D11C2001F09FFDE066BB59D86EE9
:109F100000286FD01022290001F036FDBB590498AB
:109F2000DC6EFFF705FC0D22A076BB595A706EE778
:109F3000E06E00285ED063780D2B5BD12B88082261
:109F40000382A91C123001F01FFDBB599A68517D94
:109F50000222114226D0186A407B104222D00C32D5
:109F6000E4E763780E2B45D1236F002B03D1162035
:109F700001F06AFD2067BB59186F002803D010223A
:109F8000290001F001FD0F22BB59CFE763780F2BA9
:109F900030D1206F0622691C103001F0F5FCBB594E
:109FA0009A68517D0422114203D0196A497B1142FB
:109FB000D5D100210498FFF78BFA28E7636F002BB7
:109FC0000DD0BB59586F0028F3D01022290001F0A2
:109FD000DBFC0122BB5952425B6F1A61E9E7142096
:109FE00001F032FDBB5960675B6F002BE9D126E7BA
:109FF0002978DFE707200BE76460FF1F10B5064CE8
:10A00000207001F0D1FB06212078FDF791FF034875
:10A01000FEF778FC10BDC0467760FF1F9D910011D0
:10A0200000200BB270B50D00834216DA264B18786B
:10A0300001F03AFD041E0DD00378922B0ED0A02B18
:10A0400037D0224B1878FF283AD0210001F09CFD30
:10A05000002835D180200002684070BD43780E2B67
:10A060000BD03E2BEDD18378052B12D0082BE8D1F5
:10A0700081798088FFF7D8FA08E0154B82889A42E8
:10A08000DFD183681878591CFEF7C0FE002817D16D
:10A09000D7E7104B1B785B0712D50F4B1B68002BC3
:10A0A0000ED09B68002B0BD0C289811D80889847F9
:10A0B000ECE7FFF741FAA068002801D001F05CFB53
:10A0C000200001F079FCC5E77760FF1FA93DFF1F65
:10A0D00018200000F15EFF1F6060FF1F10B50078C0
:10A0E000FFF712FA10BD10B50078FFF7FDFA10BDAA
:10A0F0000C234343084A10B59B185A68002A03D022
:10A10000012901D1904710BD9B68002BFBD000298D
:10A11000F9D19847F7E7C0469460FF1F01238340B9
:10A12000094A10B5946B1C439463506B9843506379
:10A13000D46B20009843012901D120001843D0633B
:10A14000116B0B43136310BD00800040F0B5002479
:10A150000127154B85B0DA6B144E03921A6C0192ED
:10A16000DA64019BE3403B4217D0039DE5403D404C
:10A170000295E5B202992800FFF7BAFF316A736AC7
:10A18000002908D03900002B01D00299794028001D
:10A19000FFF7C4FF01E0002BF9D101340C36172C76
:10A1A000DFD105B0F0BDC046008000407860FF1FE1
:10A1B000064B01215A68C2400A4204D01B68C340C2
:10A1C0001800084070471B6DF9E7C046008000404A
:10A1D0000122064B8240002903D0D9680A43DA6085
:10A1E0007047D9689143D960FAE7C046003800400B
:10A1F00030B5032444430F4BE25C1B199C785D7817
:10A2000001232D1B0135AB40013BA340A140DB43A3
:10A210000C00122807D808499200521811681940FA
:10A220002143116030BD054A11680B402343136080
:10A23000F8E7C0463BBE001108F0004014F00040B3
:10A24000C21F70B5D4B20623092C0BD80125084CC7
:10A250009540002908D00021FFF7CAFF23682B434F
:10A2600023600023180070BD2368AB43F8E7C046A5
:10A2700000380040214BF0B51B185B78022B21D130
:10A28000032444431E4A1F4EA35C121994780122F2
:10A2900015008540B76B013CE4B23D43A240B56375
:10A2A000194C122815D89B0000290CD117495B18AE
:10A2B00099680A439A600123205C154A834011681B
:10A2C0000B431360F0BD11495B1899689143996085
:10A2D000F1E70E4B00290DD159690A435A61225CFE
:10A2E0001328E8D00123203A93400A490868034321
:10A2F0000B60E7E7596991435961F0E77860FF1F08
:10A300003BBE00110080004080BE001100F0004004
:10A31000A0F00040A4F00040F8B500241B4E1C4DF6
:10A320001C4B1B5D012B1FD1194A9269E2401A4256
:10A330000BD00122B25693402200143AD2B2022A24
:10A3400009D815494A6913434B61013402360C356B
:10A35000172CE5D1F8BD0022B2560F4992005218D1
:10A3600091680B439360F0E7022BEED1E7B238001F
:10A37000FFF71EFF01235840C1B23800FFF77AFFF4
:10A380003800FFF715FF6877DFE7C0460DBE001104
:10A390007860FF1F7960FF1F00F000400122023843
:10A3A0008240054B002903D059690A435A6170471E
:10A3B000596991435961FAE700380040F8B50E0039
:10A3C00001210F008740114A0400D368FD43BB43BD
:10A3D000D360831E8B4201D8FFF7E0FF00212000ED
:10A3E000FFF72EFF0A4A0B4B5168012E05D1394366
:10A3F0001B1951605E700020F8BD29405160022297
:10A400001C1962709A6915409D61F4E7003800409C
:10A41000008000407860FF1F012210B58240074B8A
:10A42000002906D019680A431A600121FFF7C6FF08
:10A4300010BD196891431960F7E7C04600800040DD
:10A440000C2370B5002543430A4A29009B181D7050
:10A45000094B04001B185D70FFF7B0FF0123A340F8
:10A46000064928000A681A430A6005490A689A439F
:10A470000A6070BD9460FF1F7860FF1F3480004049
:10A480003080004070B504000E00FF2813D0032573
:10A490000540FFF7D5FF084AA3089B009B183F2201
:10A4A000ED00AA40AE401968200091433143196085
:10A4B0000121FFF78DFE70BD18380040F8B50C245F
:10A4C0004443134B0500E4186368002B03D1A368D1
:10A4D0001220002B1AD0022201270E4B00215B19FB
:10A4E0005A7028002770FFF769FF63681E1E08D0A6
:10A4F000A3683E00002B04D02800FFF759FE464019
:10A50000F6B228003100FFF709FE0020F8BDC04672
:10A510009460FF1F7860FF1FF7B5C420FF222B4B0C
:10A5200080001958002491433F3A0A431A50802270
:10A53000274F5202274E1A60274B1D5D002D21D058
:10A54000A31E012B03D80121E0B2FFF727FF012D45
:10A5500018D11F4B9B69E3402B4213D0E3B2180084
:10A560000193FFF725FE01000198FFF755FFE3B2C5
:10A57000143B022B1DD801217156184A8D40536996
:10A58000AB4353613B7F002B0DD0E5B22800FFF7B2
:10A5900095FF2800FFF70CFE7B7F0100834202D06D
:10A5A0002800FFF7A5FD01340C370236172CC3D164
:10A5B000F7BD012100237156F3568D40074A9B00D9
:10A5C0009B189A68AA439A60DCE7C04600E100E065
:10A5D0007860FF1F0DBE00117960FF1F00F0004082
:10A5E00070B50E0015000400FFF72AFF0C2363432B
:10A5F000094A20009B189D605E60FFF75FFFF02115
:10A60000064B074A8900051E5A5002D02000FFF76A
:10A6100017FF280070BDC0469460FF1F0000FF1F99
:10A620004DA1001170B5134D07202C78002C1FD1BF
:10A63000982221005200280001F09EFA0123C42034
:10A64000FF222B700C4B80001C635C630B4B1C6067
:10A650005C600B4B195891433F3A0A431A508022D1
:10A6600052021A600D20074A074901F08DF82000B8
:10A6700070BDC0467860FF1F00800040A0F0004021
:10A6800000E100E019A5001119A3001170B51D002B
:10A6900002240C2910D8094ACA40D2070CD5FBF76E
:10A6A00057FF041E08D1059A04992800FBF76CFF98
:10A6B000FCF7DAFDFFF73AFB200070BD1210000036
:10A6C00030B50D7802232C009C43184201D02B4357
:10A6D0001C0008252300AB43284201D02B00234354
:10A6E00020241D00A543204201D01C4325002A231D
:10A6F0000D70184204D011781E3B0B43137030BD0F
:10A700000028FCD10C2113788B43F7E7F8B51D0026
:10A7100006AB1B88140007AA0E000B201778002B2D
:10A7200027D10A78022A49D14A6850781178000264
:10A73000244A08438018042840D800F0E5FF03129B
:10A740001D1B2300F06801F0D7F8021CC0B2B8420C
:10A7500000D93A1CD2B22000F1682A8001F014F925
:10A7600006E00222F3681B882A8023701B0A6370AC
:10A770000020F8BD0622EEE701232B80F3681B784A
:10A780002370F5E7F368002B16D008222A801A8878
:10A7900022701A88120A62705A88A2705A88120AA5
:10A7A000E2709A8822719A88120A6271DA88A2711C
:10A7B000DB881B0AE371DBE72B80D9E701202B80C4
:10A7C000D7E7C04600D6FFFFF7B516000A781D0090
:10A7D00008AB1F880C000123022A18D14A68507860
:10A7E000117800022B4A0843801803280FD800F084
:10A7F0008BFF02254439E06801F07EF8C0B20723E0
:10A80000B84204D37B190193152B02DD0D231800E8
:10A81000FEBDE0682A003100C01901F0B5F86B46B2
:10A8200000209B88E268D0541B4B1B68834203D0F6
:10A830001B68834200D098470023E8E70B23002FD2
:10A84000E5D1022DE2D1737832781B021343E2681E
:10A850001380114B1B68002BEED01B68002BEBD034
:10A860000120E8E70B23002FD1D1062DCED12A00FD
:10A870003100E06801F088F8DEE70B23002FC6D135
:10A88000012DC3D132787533012AC0D8E3681A701C
:10A89000D2E7C04600D6FFFF8462FF1F70B50C00F0
:10A8A0001500072837D800F02FFF041436361B3662
:10A8B000242E182015290BD8184E162200213000FE
:10A8C00001F0A2F822002900300001F05DF800201C
:10A8D00070BD18200229FBD11288114B1A80F6E7AF
:10A8E00018200829F4D10A000E48290001F0ECF8DC
:10A8F000EDE718200129EBD10B4B10780B49DA69F1
:10A90000FFF7DEFEE3E718200129E1D1064B1078BE
:10A910000749DA6BF4E70220DAE7C0466C62FF1FF2
:10A92000523EFF1F483EFF1FD83DFF1F003EFF1F46
:10A93000203EFF1F030010B50020DB0704D50721D0
:10A94000024A034800F08CF810BDC04698BE0011C2
:10A95000D83DFF1F054A03001068002803D08288F5
:10A960009A4201D1806870470068F6E77C64FF1F57
:10A970000A88030008009A4204D08A8804309A4268
:10A9800000D0002070470000F8B5F22200230D4FE0
:10A990000D4E7968050042433370994200D07B60C8
:10A9A0000A4C0021200001F02FF800231A007C60DF
:10A9B000AB4202D100203370F8BD01332280DBB2FC
:10A9C000F234F5E77465FF1F7265FF1F8064FF1F97
:10A9D00073B56B4601900600684615001980FCF7B8
:10A9E00075FF041E11D1002D0FD07689002E11D0D5
:10A9F0000C2001F029F800280ED0084A04601368E2
:10AA000086808560002B02D11060200076BD1A0080
:10AA10001B68F7E70224F8E71324F6E77C64FF1FBE
:10AA2000012100220A4B10B549420A4C1980998035
:10AA30009A719A70084B2070012019805A60FFF7B4
:10AA4000A3FF2078FCF7A0FF0448FDF75BFF10BDD3
:10AA50008C62FF1F7C65FF1F7465FF1F0DAB00112B
:10AA6000022310B5002802D0FFF7B2FF0300180040
:10AA700010BD0000030010B50020DB0704D5042141
:10AA8000024A0348FFF7A4FF10BDC046ACBE001148
:10AA9000583EFF1FF0B50E2687B003930CAB1F88FE
:10AAA00002ABF6180500080031000292FDF790F89D
:10AAB00004000120002C0FD03088FFF74BFF03006B
:10AAC0000E20002B08D05E68002E05D02100280043
:10AAD000039B029A0097B04707B0F0BD0A4B10B530
:10AAE000984207D10122002352420A808B708A804B
:10AAF0008B7110BDFFF73CFF0028FAD001235B42A9
:10AB0000038000238370F4E7FFFF0000F8B5050021
:10AB100001290AD1134E00243388F227AB4219D001
:10AB200028001149FFF7DAFF06E0022904D10139B4
:10AB3000FDF766FF0028EDD0F8BD3B006343726867
:10AB4000D018D35A002B09D03A00002100F05CFF46
:10AB50000134E4B2054B1B78A342EED801235B42DB
:10AB60003380DDE77465FF1F8C62FF1F7265FF1F76
:10AB700010B5FFF7FDFE03000020834200D0987857
:10AB800010BD0000F0B589B01C000EAB80CB039067
:10AB90001E8810AB1B78049202930B7A0D00DB0623
:10ABA00016D42B780593022B24D00498FFF7D2FEFD
:10ABB000002812D003689C46002B0ED0029B220076
:10ABC000019329003B00644603980096A04705E0E6
:10ABD0000498FFF7BFFE002802D10E2009B0F0BD97
:10ABE0008368002BF9D00A2229000398984700288F
:10ABF000D7D0F3E76B6858781A786B4B0002104394
:10AC00009842D2D8043B984210D2684B984242D026
:10AC100015D8674BC0180128C7D80B20002EDDD1EE
:10AC2000EB681A7859683A80200028E0614BC01818
:10AC3000032800D979E000F067FD846A789E5E4BB6
:10AC40009842B2D10B20002EC8D101233B80EB6883
:10AC500031001B7823706889013080B2FCF7B8FF9F
:10AC60003A88031E0ED0017802328A183A8042894F
:10AC700062704289120AA27059680278E01C00F0E2
:10AC800083FE06E004323A8031000422601C00F0AA
:10AC9000BBFE0020A2E70B20002E9FD1EB6807A986
:10ACA0001E8804233B80330A300026706370FCF753
:10ACB0008FFF051E28D004AB9A890E2304A95B18C8
:10ACC0003E49C668FCF7F8FF00280BD12B783C48BA
:10ACD0006A680599FBF7AEFB002803D1012304AA9B
:10ACE0005B42D3813278022A06D17168201D00F0C0
:10ACF0004BFE3B8802333B800E2304AA9B181B8823
:10AD0000A3701B0AE370C4E704ABDE81F4E70B20F9
:10AD1000002E00D062E7E9680398FFF729FF0223BD
:10AD20003B802070000A6070B3E70B20002E00D03B
:10AD300054E70222EB681B883A8023701B0A637079
:10AD4000A7E7E86800F0D8FDC2B203000720B242CE
:10AD500000D243E70DD00299DBB27118994202DBB1
:10AD6000921BD3B20293029BE9681A003B808919B7
:10AD70005AE70023F6E70B20002E00D02EE707222B
:10AD8000EB683A801A7822705A7862705A88A270FA
:10AD90005A88120AE2701A792271DA886271DB88A5
:10ADA0001B0AA37175E7C0460429000002280000B1
:10ADB00000D8FFFFFFD6FFFF03280000FFFF0000C1
:10ADC000DCBD0011F0B58DB06B460020089120224B
:10ADD0009B5E83423DDAA64B187800F065FE071EA5
:10ADE00032D00378B02B2CD10079023816281FD826
:10ADF00000F0DAFB17001E001E001E0031001E00CE
:10AE000096001E001D011E0052011E0073011E004F
:10AE1000CD011E0050021E001E001E008E021E00EC
:10AE2000E302944B94491B8878880B80FBF742F827
:10AE30003800FCF7C3FF914B1B68002B01D0380092
:10AE40009847380000F0B8FD8020089B000243407E
:10AE500018000DB0F0BDEE220021874800F0D4FDAF
:10AE60000BAA3B7B7989388900923A000D32FCF7B6
:10AE7000C7FD0400804B1B78002C3FD146E0804B7F
:10AE8000788805937F4B4100CB5A0BAE073BDBB272
:10AE900032880293002301937B4B21000693009399
:10AEA000059BFFF76FFE744D002810D1069B3A8A70
:10AEB0001B889A420BD138000599123000F0F4FB40
:10AEC000002804D02B7862899B00EB185A80162347
:10AED00006A81B18328820007989FCF7EDFE2B7834
:10AEE00004009A00AA1851880029C3D00133DBB2AC
:10AEF0002B70002807D006A9C98A9180634A12885E
:10AF00009A42BCD802E0012149429180002B04D032
:10AF100059497888FBF702F88AE73E890A2479E0E4
:10AF200000253E89574B06937B88069A5B009B5A07
:10AF3000033B9D4202DB002DF0D05BE0162206A809
:10AF400012183B7B798900923A0030000D32FCF7F1
:10AF500057FD0590002858D04689017A7888FCF77B
:10AF600019FD041E44D1464B78880793069B410087
:10AF7000C95A454B0439C9B206AAD28A069302912E
:10AF8000019400930599079BFFF7FCFD041E2FD148
:10AF9000069B39491A88931C002D26D14B8079884D
:10AFA000384B4900CB5A5119033B8B4220DD059B9E
:10AFB00031485B8941190B71A91C0135C9B2EDB249
:10AFC000059145191B0A2B71059B2D49043318184F
:10AFD00000F0DAFC2C4B059A1B88D318DDB22C4B01
:10AFE0009E4205D00136B6B29CE749889942D6D038
:10AFF000002D0CD0204C2800618800F0E5FC20706A
:10B0000021007888FAF79AFF12E7059CF0E7002CF8
:10B0100000D183E77B78142B00D109E716493B79EF
:10B020004E800B700C717888FAF73AFF00E716240F
:10B0300006ABE41821003889FCF7CAFD011E00D1D7
:10B04000B7E1788822880F4C45002C5B0A4D013C03
:10B05000E4B2029400240F4B01940095FFF792FD97
:10B06000041E00D014E129007888FAF777FFDFE6A4
:10B070007C65FF1F483DFF1F9462FF1F8862FF1F12
:10B080008863FF1FC45EFF1F7864FF1F463DFF1FDC
:10B09000FFFF00009662FF1F162406ABE418210094
:10B0A0003889FCF795FD011E00D182E1788822885D
:10B0B000AE4C45002C5BAE4D013CE4B202947C8961
:10B0C000AC4B01940095FFF75DFD041E00D0DFE05E
:10B0D00029007888FAF74CFFAAE60025A44B1D80CA
:10B0E0003B00F6331B78A24A78880792AB4208D916
:10B0F0009E4B12880693069943005B5A013B9A4285
:10B1000003DB0799FAF73EFF92E616246B00FB1863
:10B11000059306ABE418059B21001889FCF758FD40
:10B12000011E03D1059B01241E8973E77888924B89
:10B130002288069C099343001B5B904E013BDBB2C7
:10B140000293002300960193099BFFF71BFD041E49
:10B1500002D0059B1E895DE77B88069A5B009B5A9F
:10B16000079A108832881218934202DC1B1A013B9E
:10B1700033807F4C023032880999001900F004FCBA
:10B180002388328801359B182380EDB2A8E70BAAEB
:10B190003B7B7989388900923A000D32FCF730FC0C
:10B1A00000250590059B002B04D10A24002D00D119
:10B1B0006EE060E0059B7888197AFCF7EBFB0100F4
:10B1C000041E63D1694C6C4B788806940993069BE6
:10B1D0004400E45A694B063CE4B20BAE3288079354
:10B1E0000294019100930599099BFFF7CBFC041E83
:10B1F0004CD1079B5E491B881A1D002D30D14A8017
:10B20000059B5B4C5A8963191A716B1C9BB2E3183E
:10B21000120A1A71162306A832881B187989059814
:10B22000FCF74AFDFF21AA1C2E1D03350B000590DB
:10B2300092B2B6B2ADB2002803D006ABDB8AD9B267
:10B240001B0AA218651911712B714C4D301D2A88EB
:10B250004949201800F098FB2B88F618B5B2A1E7F1
:10B260004988914207D17A8806995200525AEB18C0
:10B27000053A9A42C4DC3E4C2800618800F004FC88
:10B28000207021007888FAF787FED1E5002DF2D1F1
:10B290003E89BFE6162606ABF61831003889FCF762
:10B2A00097FC3D000400FA3500282DD0037A9B0658
:10B2B0000CD400227B893989788800923A000C32BC
:10B2C000FFF7E8FB041E10D03E8915E03088FFF739
:10B2D00041FB00281AD08368002B17D021001222CE
:10B2E00078889847041EE4D0EEE72B78002B02D133
:10B2F0007888FAF761FE00262B78002B00D097E5BE
:10B30000002C00D194E585E60124DDE70E24DBE77F
:10B31000162506ABED1829003889FCF759FC041EE8
:10B3200047D0037A9B0611D4154A7B88118899422D
:10B3300003D01448814207D11380134BF2261D78A5
:10B340000023D9B2A94221D30924A1E72888FFF715
:10B3500001FB00282FD08368002B2CD02100122263
:10B3600078889847041EDFD092E7C046C45EFF1F6E
:10B370009462FF1F9662FF1F8863FF1F7864FF1FA0
:10B380007465FF1FFFFF00007265FF1F3100594306
:10B39000546801336018615A0029D2D13C00083446
:10B3A0002100F22200F0F0FA21007888FAF70CFE72
:10B3B0003EE501246CE70E246AE71D4B1A887B8862
:10B3C0009A4231D07888FAF709FE31E5F2230598E0
:10B3D00051684343CD18C95A00291FD03B7A012B2D
:10B3E0000BD16C88AB887888AA1D0094FFF752FBBC
:10B3F000041E02D000233B722E88F2220021280076
:10B4000000F002FB00232B80059B0133DBB2059388
:10B41000084B05991B78064A8B42D7D801235B421B
:10B420001380002CCED0F5E5002634000596EFE71A
:10B430007465FF1F7265FF1F70B504000E001500D4
:10B44000FFF796FA031E08D131000548FFF790FA7E
:10B4500003001120002B02D01C8000209D7070BDC5
:10B46000FFFF0000F8B50B4F06003B780D001400FD
:10B47000FF2B0ED00A2000F027FA011E09D0B123BD
:10B480000380002346800371C5800481387800F072
:10B490007BFBF8BD993EFF1FF7B50F0008A906001A
:10B4A000088809A90B240988002821D10234022B1D
:10B4B0001ED1557813782D021D432B008B43019329
:10B4C0007334002B14D1FB68300019000093FFF790
:10B4D0004FFB019C85420BD02A0030000099FFF7FA
:10B4E000ABFF041E04D12A0030007989FFF7BAFFB0
:10B4F0002000FEBDF0B50E7885B003900AA805883F
:10B500000120022E0DD14C682778647824023C4338
:10B51000054FBC4205D10398DBB201960095FFF7B9
:10B52000BBFF05B0F0BDC04602290000034B10B5BB
:10B530001B68002B00D09847FEE7C0468065FF1FC0
:10B5400007B501A8FFF7F2FF044A05480021121AC7
:10B5500000F012FBF8F74EF9FEE7C0468465FF1FC6
:10B560009C3EFF1F0000000001B40248844601BC5D
:10B57000604700BF492DFF1F01B40248844601BC4B
:10B58000604700BF75A9000001B40248844601BCB1
:10B59000604700BF8552010001B40248844601BCE7
:10B5A000604700BF350E000001B40248844601BC6C
:10B5B000604700BF6136FF1F01B40248844601BCEA
:10B5C000604700BF0124000001B40248844601BC6A
:10B5D000604700BF017F000001B40248844601BCFF
:10B5E000604700BF3936FF1F01B40248844601BCE2
:10B5F000604700BFF92AFF1F01B40248844601BC1E
:10B60000604700BFE528FF1F01B40248844601BC23
:10B61000604700BF0D52010001B40248844601BCDE
:10B62000604700BFC94A010001B40248844601BC1A
:10B63000604700BF2124000001B40248844601BCD9
:10B64000604700BF056A000001B40248844601BC9F
:10B65000604700BFED4A010001B40248844601BCC6
:10B66000604700BFD91B000001B40248844601BCFA
:10B67000604700BF2146010001B40248844601BC76
:10B68000604700BF5952010001B40248844601BC22
:10B69000604700BFB352010001B40248844601BCB8
:10B6A000604700BF9134FF1F01B40248844601BCCB
:10B6B000604700BFCD4C010001B40248844601BC84
:10B6C000604700BF5118FF1F01B40248844601BC07
:10B6D000604700BFC9A9000001B40248844601BC0C
:10B6E000604700BF5933FF1F01B40248844601BCC4
:10B6F000604700BFA54F010001B40248844601BC69
:10B70000604700BF6DBC000001B40248844601BC24
:10B71000604700BF4D36FF1F01B40248844601BC9C
:10B72000604700BF3D18000001B40248844601BCD8
:10B73000604700BF1147010001B40248844601BCC4
:10B74000604700BFDD66010001B40248844601BCC9
:10B75000604700BF014C010001B40248844601BCAF
:10B76000604700BF7D18FF1F01B40248844601BC3A
:10B77000604700BFC56D010001B40248844601BCAA
:10B78000604700BFD949010001B40248844601BCAA
:10B79000604700BF812BFF1F01B40248844601BCF3
:10B7A000604700BFC51D000001B40248844601BCCB
:10B7B000604700BFC926000001B40248844601BCAE
:10B7C000604700BFE928000001B40248844601BC7C
:10B7D000604700BF5D17000001B40248844601BC09
:10B7E000604700BFE12AFF1F01B40248844601BC44
:10B7F000604700BF0D35FF1F01B40248844601BCFD
:10B80000604700BF6571010001B40248844601BC75
:10B81000604700BF291C000001B40248844601BCF7
:10B82000604700BF5522000001B40248844601BCB5
:10B83000604700BFB54C010001B40248844601BC1A
:10B84000604700BFF30E000001B40248844601BC0B
:10B85000604700BF090E000001B40248844601BCE5
:10B86000604700BF3555000001B40248844601BC62
:10B87000604700BF5125000001B40248844601BC66
:10B88000604700BF691F000001B40248844601BC44
:10B89000604700BF456B010001B40248844601BC0B
:10B8A000604700BF851F000001B40248844601BC08
:10B8B000604700BF091B000001B40248844601BC78
:10B8C000604700BF2951010001B40248844601BC11
:10B8D000604700BF1D4D010001B40248844601BC11
:10B8E000604700BF4D1F000001B40248844601BC00
:10B8F000604700BFA533FF1F01B40248844601BC66
:10B90000604700BFDD52010001B40248844601BC1B
:10B91000604700BF212DFF1F01B40248844601BCCF
:10B92000604700BF8B52010001B40248844601BC4D
:10B93000604700BFADAE000001B40248844601BCC0
:10B94000604700BF156B010001B40248844601BC8A
:10B95000604700BF2534FF1F01B40248844601BC84
:10B96000604700BF9DA9000001B40248844601BCA5
:10B97000604700BF6D33FF1F01B40248844601BC1D
:10B98000604700BF6532FF1F01B40248844601BC16
:10B99000604700BFE94C010001B40248844601BC85
:10B9A000604700BFB14E000001B40248844601BCAC
:10B9B000604700BFBD30FF1F01B40248844601BC90
:10B9C000604700BF434D010001B40248844601BCFA
:10B9D000604700BF350E000001B40248844601BC38
:10B9E000604700BFE548000001B40248844601BC3E
:10B9F000604700BF7918000001B40248844601BCCA
:10BA0000604700BFA946010001B40248844601BC5A
:10BA1000604700BF154D010001B40248844601BCD7
:10BA2000604700BFB130FF1F01B40248844601BC2B
:10BA3000604700BFEDA5000001B40248844601BC88
:10BA4000604700BF311B000001B40248844601BCBE
:10BA5000604700BF3D4B010001B40248844601BC71
:10BA6000604700BFE117000001B40248844601BCF2
:10BA7000604700BF3935FF1F01B40248844601BC4E
:10BA8000604700BFE130FF1F01B40248844601BC9B
:10BA9000604700BF090E000001B40248844601BCA3
:10BAA000604700BF8D12000001B40248844601BC0B
:10BAB000604700BFF54E010001B40248844601BC56
:10BAC000604700BF2526000001B40248844601BC3F
:10BAD000604700BF810E000001B40248844601BCEB
:10BAE000604700BF055E000001B40248844601BC07
:10BAF000604700BF5549010001B40248844601BCBB
:10BB0000604700BF792EFF1F01B40248844601BC84
:10BB1000604700BFF94C010001B40248844601BCF3
:10BB2000604700BF4550000001B40248844601BC94
:10BB3000604700BFB131FF1F01B40248844601BC19
:10BB4000604700BF5147010001B40248844601BC70
:10BB5000604700BF392BFF1F01B40248844601BC77
:10BB6000604700BF4551010001B40248844601BC52
:10BB7000604700BF1D4B010001B40248844601BC70
:10BB8000604700BFB70E000001B40248844601BC04
:10BB9000604700BF594F010001B40248844601BC10
:10BBA000604700BFC521000001B40248844601BCC3
:08BBB000604700BFE533FF1FF1
:10BBB8000003010202030303040305000602070051
:10BBC800080209030A030B030C000D000E030F0300
:10BBD800100311031303140315021602B13B0011DD
:10BBE800E53B00110000000002000000FABB001154
:10BBF800192A0F180A000000F1590000FD2400005E
:10BC0800414601000D80001121A00011757400113A
:10BC1800117E0011ED520011C5AD0011554F0011F4
:10BC2800A53D0011D53E00110000000016160000C9
:10BC38000200000044BC0011F4FFF3FFD2FC000036
:10BC480015400011000000000000000054757961E3
:10BC58000042312E3400303031370067697468751E
:10BC6800622E636F6D2F70767678005448423100EB
:10BC7800020000008CBC0011292A282A272A262A1B
:10BC8800252A242A0A180000E20400007102000094
:10BC980078EC0000744000001027000060F00000FD
:10BCA80006640000204E00000000000005000000AF
:10BCB8001F501D00023CB4000001170014000000D2
:10BCC800A102000030313233343536373839414239
:10BCD8004344454600000000F15600114557001145
:10BCE8000000000002000000F8BC00116F2A6E2A54
:10BCF8001A18EAD8BC80F0FC6000000000000000C0
:10BD080000005F066B2F363D7D077F3F777C596EBD
:10BD18007971000001A00000000000006410B71D48
:10BD2800C8206E3BAC30D9269041DC76F4516B6B61
:10BD38005861B24D3C7105502083B8ED44930FF023
:10BD4800E8A3D6D68CB361CBB0C2649BD4D2D386D9
:10BD580078E20AA01CF2BDBDFB349B5F8000008026
:10BD6800001000000000000077600011017700114A
:10BD78009B600011097B00111F610011DF7A00111F
:10BD880095610011B57A0011E76100117D7C001101
:10BD98004F6200117D7C001181620011377C001117
:10BDA800956100116D7A00110D620011157C00116A
:10BDB8000000000000000000F3620011157C001173
:10BDC8005563001119770011052A042A012A002A4F
:10BDD8000229032801280028011800180000000083
:10BDE80000000000000000000000008701010201BF
:10BDF800020101020102030304010301010101011F
:10BE08000303020103000D000E00100011001300CF
:10BE18001401070108010A010B011C011D0204029B
:10BE280005020702080219021A021C021D03010377
:10BE3800020317000201000504000807000B0A00AE
:10BE48001716001D1C010201010504010E0D011148
:10BE580010011413011716011A19020201020B0A24
:10BE6800020E0D0211100214130217160305040323
:10BE78000807030B0A030E0D0001020307090A0B4A
:10BE88000E0F101112141718191A1B1F2021220047
:10BE98000DA70011C9A70011000000000200000052
:10BEA800E2BD001100000000F5B400110000000020
:08BEB80002000000E0BD0011D2
:020000041FFFDC
:10000000000000000D3D001100BC0011FCBB001100
:10001000A85BFF1F000000000000000000000000BF
:1000200000000000000000000000000000000000D0
:1000300000000000000000000000000000000000C0
:1000400000000000000000000000000000000000B0
:1000500000000000000000000000000000000000A0
:100060000000000000000000000000000000000090
:100070000000000000000000000000000000000080
:100080000000000000000000000000000000000070
:100090000000000000000000000000000000000060
:1000A0000000000000000000000000000000000050
:1000B0000000000000000000000000000000000040
:1000C0000000000000000000000000000000000030
:1000D0000000000000000000000000000000000020
:1000E0000000000000000000000000000000000010
:1000F0000000000000000000000000000000000000
:1001000000000000000000000000000000000000EF
:1001100000000000000000000000000000000000DF
:1001200000000000000000000000000000000000CF
:1001300000000000000000000000000000000000BF
:1001400000000000000000000000000000000000AF
:10015000000000000000000000000000000000009F
:10016000000000000000000000000000000000008F
:10017000000000000000000000000000000000007F
:10018000000000000000000000000000000000006F
:100190006D2DFF1FCD2BFF1FC16601000000000069
:1001A000000000000000000000000000000000004F
:1001B000000000000000000000000000000000003F
:1001C000000000000000000000000000000000002F
:1001D000000000000000000000000000000000001F
:1001E000000000000000000000000000000000000F
:1001F00000000000000000000000000000000000FF
:1002000000000000000000000000000000000000EE
:1002100000000000000000000000000000000000DE
:1002200000000000000000000000000000000000CE
:1002300000000000000000000000000000000000BE
:1002400000000000000000000000000000000000AE
:10025000000000000000000000000000000000009E
:10026000000000000000000000000000000000008E
:10027000000000000000000000000000000000007E
:10028000000000000000000000000000000000006E
:10029000000000000000000000000000000000005E
:1002A000000000000000000000000000000000004E
:1002B000000000000000000000000000000000003E
:1002C000000000000000000000000000000000002E
:1002D000000000000000000000000000000000001E
:1002E000000000000000000000000000000000000E
:1002F00000000000000000000000000000000000FE
:1003000000000000000000000000000000000000ED
:1003100000000000000000000000000000000000DD
:1003200000000000000000000000000000000000CD
:1003300000000000000000000000000000000000BD
:1003400000000000000000000000000000000000AD
:10035000000000000000000000000000000000009D
:10036000000000000000000000000000000000008D
:1003700041B5001100000000000000000000000076
:10038000000000000000000000000000000000006D
:10039000000000000000000000000000000000005D
:1003A000000000000000000000000000591AFF1FBC
:1003B000000000000000000000000000000000003D
:1003C000000000000000000000000000000000002D
:1003D000000000000000000000000000000000001D
:1003E000000000000000000000000000000000000D
:1003F00000000000000000000000000000000000FD
:081838009069FF1F4118FF1F1A
:10184000024981F3088801F01FFF00009069FF1F23
:1018500010B502F0A1F8072804D0122808D00228F9
:1018600008D010BD044A0420136B01331363F8E75A
:101870000220F6E71420F4E76C5FFF1FF8B50700BD
:101880000C0026002500503630785135002804D150
:101890000300287058342370F8BD2978CA00481E08
:1018A0008141A3183800A25C5B68C9B2FFF7D0FF82
:1018B00000280DD12B78DA00A218013350602B706C
:1018C0003378044A013B3370136A01331362D8E75B
:1018D0000123DFE76C5FFF1F5C234343074910B51B
:1018E000C9180B0058331B78012B05D1FFF7C6FF31
:1018F000034A936A0133936210BDC046A05FFF1F85
:101900006C5FFF1F10B502F07FF8064A012113003B
:1019100010CB4942D967044B136001F05DFF2000F2
:1019200010BDC04600E100E01000100010B504003A
:1019300002F06AF8024B1C6001F04EFF10BDC04679
:1019400000E100E0431E5A425341A022F0B5D2010B
:101950005B421340154D164A40019B182A18127E0F
:101960008BB00191002A1BD01A000832D46F0022DC
:10197000E6B206AFE4B294420EDC2818C369002B2D
:1019800008D0019902AA117106AA049202AA16733C
:1019900003A898470BB0F0BD1978B9540132EAE7B3
:1019A0001A7D1A7806AB01261A70E6E72C62FF1F33
:1019B00000400040F0B5254B04004001C25C85B0FA
:1019C000002A2BD01A18117E002927D0917E0029D9
:1019D00024D01179022921D11689D788D168F51B25
:1019E000ADB22A1C102D00D9102292B2BE4217D1DE
:1019F0001818012303710023C269C38003819A422E
:101A000006D06846032103730171029301A8904731
:101A10000820002C00D0192001F08EF805B0F0BD90
:101A2000013C65426C41A0256442ED012C40084D0B
:101A30001B186419074D0633013A92B2AA42EDD041
:101A40001888461C1E80085C2070F5E72C62FF1F7A
:101A500000400040FFFF00000F220E4B10B59868B9
:101A6000104002380A280BD801F0F0FD0D0A0B0ACD
:101A70000A110A0A0A0A060002210020FFF762FF83
:101A800010BD0121F9E70020FFF794FFF8E7DB6FB5
:101A9000F6E7C046004000400F220E4B10B5986894
:101AA000104002380A280BD801F0D0FD0E0A0B0AAC
:101AB0000A120A0A0A0A060002210120FFF742FF61
:101AC00010BD01210800F9E70120FFF773FFF7E7D8
:101AD000DB6FF5E700900040564B70B51B68012B9B
:101AE00003D1554A936D0133936501F04DFE534B7D
:101AF000534A1860534B544C1A600123534A1360E5
:101B0000534A13602378002B06D0062251495248CD
:101B100001F04AFE00232370504A514B10681B7895
:101B2000C1B2002B0ED14F4CC0B223785BB2002B58
:101B30004FDB237824785BB264B21B0424021B19A8
:101B40001B1813600B1C50294ED95023464A474995
:101B50001078DBB2FF2202284BD10868444C454D77
:101B6000267890432A78964254D9227824782E7881
:101B7000023B5D10A31B6B435201D31A10335B1160
:101B80001843086001F078FF031F012B45D83A4B3A
:101B90001B78002B06D0394B1B78002B02D000207D
:101BA00001F082FEA122364B92009978354B4A43D0
:101BB0001B689B18832292009B181B78033B012B08
:101BC00003D8AF20400001F02FFF01222E4BDA8214
:101BD00070BD237824785BB264B2FF33FF341B04FA
:101BE00024021B190138ABE7CAB2022AAED2022383
:101BF000ACE70868254C264D267890432A78964213
:101C000008D9227824782D78023B5B10641B63434B
:101C10005201B2E72378DBB2B2E70228D5D11D4BDF
:101C20001B78013B022B03D91B4B1B78022BCCD119
:101C30006C20C8E79809FF1FFC0FFF1FA45EFF1F61
:101C4000FF3F000014100340A85EFF1F0C1003406C
:101C500000100340D50BFF1F7211FF1FB40003409B
:101C60008C09FF1F680AFF1F490AFF1F94000340E9
:101C7000460AFF1F470AFF1FF908FF1F2209FF1F1F
:101C8000300DFF1F3409FF1FBC0BFF1F440AFF1F4D
:101C9000450AFF1F1C09FF1F2309FF1F10B501F094
:101CA0009BFE0022014B1A8010BDC046A25EFF1FA2
:101CB00070B5244D2B68002B28D001F05DFE2B68F9
:101CC000D8402B680400002B27D001F0E5FD2B68DD
:101CD000D8401D4B1D4A9978A1239B004B431268A5
:101CE000D118D25C91239B00002A20D0CA5801321F
:101CF000CA50174B17491B680868834214D3D23B5C
:101D0000181A012A1AD0144B186070BD01F034FE65
:101D1000124B196801F0D8FCD3E701F0BDFD0F4B61
:101D2000196801F0D1FCD4E70D495B18E8E7CA5007
:101D30000C4B1B68DB68E418201AE4E7F530FF3031
:101D4000E1E7C0461C08FF1F300DFF1F3409FF1FCD
:101D50009C09FF1FA45EFF1FA009FF1F1808FF1F9B
:101D60002DFF3F00AC5EFF1F70B504000D00282959
:101D700016D10300A433C2881B889B1A0B4A9BB25E
:101D800093420DD906006A3605223100653001F014
:101D900093FE002804D13100200001F0E5FD70BD64
:101DA0002900200001F050FEF9E7C046FE7F000048
:101DB000F8B50500012001F0A7FD134CA36AA26A43
:101DC0009342FBD1114E336001F096FD10490300A0
:101DD00008601048426894460F4A17680022BC45C4
:101DE00001D24268BA1A0D4802603268AD18A422C6
:101DF000E562606A520302436262094A1278002A6D
:101E000001D00F3B0B60F8BD00F00040340AFF1F0B
:101E1000E408FF1F28100040180AFF1F1C0AFF1FBC
:101E20001C09FF1F70B580241025E405A3682B430F
:101E3000A36001F029FDA368AB43A36070BD00005F
:101E4000F7B5160080221C001023D205019191687D
:101E500005000B43936000225A4BD7301A6001F003
:101E60008BFC9D232A002F009B00EB58CA320121D6
:101E70000092FC37002B01D00021009A386801F055
:101E80009BFD2900009BCB311A784F4BD3351A604C
:101E90004B780A781B0213438A7812041A43CB78D2
:101EA0001B061343494A1BBA13604B790A791B027C
:101EB00013438A7912041A43CB7931001B0613436A
:101EC000434A1BBA13606B782A781B021343AA7823
:101ED00012041A43EB781B0613433E4A1BBA1360E5
:101EE000019A330213433C4A13603C4B22001B1BF4
:101EF0009C4603293DDCB3089A0013005142B21AF4
:101F0000032A46D1354AE018511A827840781204E3
:101F100000020243E05C043302430A600022FF2B0C
:101F20004BDDF0222E4B12011A600F222D4B1A604E
:101F30002D4A1368002BFCD00023224A2749136046
:101F4000091B321D0B191B68043A180A23706070B4
:101F5000180C1B0EA070E3700434002AF2DC8022FF
:101F600010213B68D20501333B6093688B4393603B
:101F7000F7BD6346D578981893782D061B042B433C
:101F8000157804392B43557804322D022B43036016
:101F9000AFE7022A0AD1114AE05C511AE2185278DE
:101FA000120202430A6004339BB2B7E7012AB5D19B
:101FB0000A4A521AE15C1160F5E7084959180A60AB
:101FC0000433ACE7000004403C0004403800044007
:101FD00034000440300004400C0004400001044080
:101FE000040004401000044014000440F7B515003C
:101FF00080221C001023D2050091916807000B433A
:1020000093600023654AD730136001F0B5FB9D2330
:102010003E009B00F9583B00CA363200FC330029D1
:1020200000D07FE0586801F0C7FC390032785C4B83
:10203000CB311A604B780A781B0213438A78AC467E
:1020400012041A43CB78281D1B061343554A1BBAAA
:1020500013604B790A791B0213438A7912041A43DD
:10206000CB791B061343504A1BBA13604B7A0A7A8A
:102070001B0213438A7A12041A43CB7A21001B06EF
:1020800013434A4A1BBA1360009A2B021343484A6F
:1020900013602200474B1B1B0093009BCE785B18FC
:1020A00001938B7836061B0433430E780438334390
:1020B0004E78043136023343019E33600328ECDC52
:1020C0000321A808431C9B002940800003292BD131
:1020D0003849E5185E18A9786D78E35C09042D028B
:1020E000294319433160030008330021FF2B2DDD04
:1020F000314B324919600F21314B196001232749B7
:102100000B60304B19680029FCD006211B680B407E
:10211000042B20D080220020D20593680A318B4303
:102120009360FEBD01217DE7022908D121495D1898
:10213000E1184978E35C090219432960D3E70129D2
:10214000D3D11C495918E35C0B60CCE71948181827
:1021500001600433CAE7002310490B606346002B7B
:102160000CDC3B00FC335A68102101325A6080229B
:10217000D205936801208B439360D2E7009B9B18A4
:102180001B68190A13705170190C1B0ED3700423AD
:102190005B4291709C440432E0E7C046000004407A
:1021A0003C00044038000440340004403000044047
:1021B0000C0004400001044004000440080F00002B
:1021C000100004401400044010B5002901D001F0B3
:1021D00063FC10BDF7B5604B01919978A1239B007A
:1021E0004B435E4A060014681022E418D6235B00B5
:1021F000E0583623FF33E35C00279343222B41D181
:10220000574B0F3A1A600760012501F09DFB019BB7
:102210001880E8235B00E35C002B01D0B34258DD5B
:102220000023504FFB70AD33FF33E3581A68002A88
:1022300003D09B88DB439B071DD03823FF33E35C2F
:10224000002B18D09B235B00E35C002B13D1D13310
:10225000FF33E35CB3420EDAA4235B00E15AE018DB
:10226000090A023101F030FB23000122FE33013E56
:1022700001351A87FA70E8235B00E35C002B2AD053
:10228000A8B2FEBD03683D00002BBED0818804309B
:10229000090A023101F018FBD6235B00E3581F60E6
:1022A000B2E72300B133BA00FF3398580137818871
:1022B0000430090A023101F007FBE8235B00E35C0C
:1022C000BB42EEDCE822F61AED1800235200A354BC
:1022D000A6E70027F1E7200001F0A6FA00281FD0AA
:1022E000002E1DDD7319882647190193B6002000C2
:1022F00001F022FB5A3080002018406801358188A7
:102300000430090A023101F0DFFA200001F094FBE9
:10231000A3590133A351BD4202D0019B9D42E6D196
:10232000114BE35C002BABD095239B00E35C002BAF
:10233000A6D00E4BE15A0029A2D00D4AA35C9942C7
:1023400002D90133A3549BE700231A212000A35490
:1023500001F062FB94E7C046300DFF1F3409FF1FF8
:1023600000140340E010FF1F5A0200007202000038
:102370005E0200000D4970B54A6E0D4CD2038B69A8
:10238000D20BA24206D80B4D0224AA4204D901F076
:10239000CBF970BD02246442E21815007E2425406A
:1023A0002242F4D0A3432B438B61F0E700F00040BE
:1023B0000A200000FC1C00000B001B3B70B5040051
:1023C0003020E02B0DD81300E025493BFF3B9BB2AA
:1023D000ED00AB4205D8034B200019825A8201F070
:1023E000BBFA70BD8410FF1FD722044B92009B588C
:1023F00010B5002B00D0984710BDC0460000FF1F4D
:1024000010B501F0ADF8FFF7EFFF2749274BCA6D74
:10241000274C1A4084235B001343CB65254B1B6874
:10242000186A01F071FA244B244A1A60244B254A99
:102430001A60A022244B52001A60244B187801F035
:1024400003FA2000224901F02FFB0023A36002338E
:10245000A360204B2049236003232048A36001F0A0
:1024600023FB10221E4BFF201A60802252031A60A9
:10247000802292031A60802212041A6001F014FA7A
:10248000012001F069F9FA20400001F0D5F9582047
:1024900001F0CAFA134801F07FF9012001F0FCF8BD
:1024A000072001F0B9F910BD00F0004000FEFEFF6A
:1024B00014100040AC5EFF1F000003400180063D89
:1024C000BC00034034080000A40003404A0AFF1F78
:1024D00071020000C3090000FFFF3F002810004008
:1024E00000E100E030750000674E336888331B68F8
:1024F00083F3088801F0C8FA644A6549136800202C
:102500000B401360634B644A1B68934200D1A6E002
:1025100001F0AAF90221614A13688B431360FFF7A7
:102520006FFF5F4B5F4C1878C0B201F0DDF80023FD
:10253000A3600233A3605C4B0120236001F0E4F947
:102540000323A36001F088FA040001F01DF90500DF
:1025500001F082FA554B186001F016FA544B1968D5
:10256000621A531EA14200D213008022D20393426A
:1025700001D39B029B0A3268D16AC90700D471E07B
:102580004C491C0C09689BB24C4359432402090A6C
:10259000641803264849FC3293680A6847489B1A26
:1025A000474A0768126847499B18474A9A183340B8
:1025B0009208DB190A600360042B03D9013233400F
:1025C0000A6003600E684149A619300001F07CF8EA
:1025D0003F4F3E493B68C3183B603000019301F018
:1025E0008BF83C4E3068081838493060884205D96D
:1025F000019B01333B6001F07FF8316001F0D4F9B9
:10260000354B1B78002B0DD001F0BEF8334B621B0D
:10261000196812188A4232D24919091B091A30481E
:1026200001F042FA2F4E337A002B0ED001F0ACF8B5
:10263000621BF1681218914224D94919091B091A21
:10264000294801F031FA00233372284B83F30888BC
:1026500001F0D2F9002001F007F901F085F801F04E
:1026600003F95CE7DC0199000234641A5900641A2A
:1026700009214B438033CB40A408E41889E7FA21B1
:102680008900CCE71A49DBE7AC5EFF1F1CF0004075
:10269000FFFFC1FF0C0AFF1FB641210310000040DD
:1026A000490AFF1F14100040C3090000100AFF1F51
:1026B000340AFF1F380AFF1F200AFF1F280AFF1FC6
:1026C0001C0AFF1F240AFF1FC4090000710200003A
:1026D0006008FF1F2C0AFF1F1C09FF1FE408FF1FD3
:1026E00000100040740BFF1F3C1000400000002051
:1026F000DC050000A022054B92009B5810B5002B72
:1027000001D0984710BD01F007F9FBE70000FF1F5B
:10271000A122054B92009B5810B5002B01D0984781
:1027200010BD01F0F9F8FBE70000FF1FA222054BE6
:1027300092009B5810B5002B01D0984710BD01F0B6
:10274000EBF8FBE70000FF1FA322054B92009B580C
:1027500010B5002B01D0984710BD01F0DDF8FBE764
:102760000000FF1FA422054B92009B5810B5002BC0
:1027700001D0984710BD01F0CFF8FBE70000FF1F24
:1027800070B501F001F84F4B186000F095FF0400A0
:10279000C30702D400F0B8FF70BD00224A4B1A6094
:1027A0004A4B18780138042829D800F04FFF03203D
:1027B000181C2400200001F08FF80128ECD0444CB4
:1027C0002378042B6ED101F057F80028E4D001F0F3
:1027D0008BF8582001F028F902232370DCE7200051
:1027E00000F07AFFE9E7200001F06EF9E5E720004C
:1027F00000F092FFE1E7200000F09EFFDDE701F02E
:102800003BF90500012808D1324B1B78053B012B11
:1028100003D82000FFF76EFFD1E72D4B1B78022B6A
:1028200001D0052B20D1022D28D12B4B9B7BAB4314
:102830001CD12000FFF76CFF264B18780128BED171
:102840006405BCD4244925224B7B034205D1233A9D
:1028500013405A42534126331A000B7D9342AED99E
:10286000322001F029F8AAE7022D07D1194B1B7875
:10287000052B11D12000FFF759FFDDE7012D0BD10A
:10288000012B03D12000FFF75FFF98E7062B03D150
:102890002000FFF767FF92E7200001F03DF8022DCE
:1028A0008DD1C9E7032B04D10C4B987C00F08CFF31
:1028B00072E7072B00D06FE7094B987B00F0DCFE36
:1028C0006AE7C0469C09FF1F9809FF1F9009FF1F78
:1028D0002309FF1F1C09FF1FA60BFF1FBC0BFF1FB7
:1028E000D40BFF1F10B500F099FE10BDF7B50B0C0F
:1028F000FF270122009300233C001E001D00944688
:10290000019089B262469A4010000840184136187A
:10291000B6B2FF2F02D1012E00D19FB20098024023
:102920001A41AD18ADB2FF2C02D1012D00D19CB2DD
:102930000133102BE6D10320012E07D1012D04D144
:10294000019B2401E4191C700138FEBD102EFCD13E
:102950000238102DF9D00230F7E700008023F7B5D8
:102960009C46264B264F01932649274A274D284C43
:10297000284B02281AD1604638600868264E30403D
:10298000802636033043086001990978002909D16F
:102990001660224A2A60224A2260E0221968914386
:1029A000A03A1BE08021C9021160F2E766463E6052
:1029B0000F68194E3E408027FF023E430E6001998A
:1029C000097800290DD1176001280ED1154A2A6017
:1029D000154A2260E02219689143C03A0A431A60FE
:1029E000F7BD802189021160EEE7E0210F4A024322
:1029F0002A600F4A22601A688A43F0E74B0AFF1FD9
:102A0000E0000340D8000340900003400000034072
:102A10005000034040000340FFFFE3FF0280063DFB
:102A2000804508220180063D8066082200800698C5
:102A300080550822F8B51E4B80261A680020140025
:102A40003440324232D11A681A4F32431A6001229E
:102A50003B68063093433B6000F056FF0122164D61
:102A60002B681E432E603B680A2613433B60802779
:102A7000BF00124B1B683B4211D1013EF6B2FF2E44
:102A800009D17E220E4B1C682B68E40B1440934343
:102A900023432B6005E0082000F036FFE9E7002E15
:102AA000EFD180222B68600893432B60F8BDC046AD
:102AB000C4F000405CF0004018F0004068F00040B6
:102AC00060F0004010B500F0C7FE01215820034A15
:102AD00000F072FEFFF7AEFF10BDC046600AFF1F98
:102AE00010B578220021034800F086FE00F0DCFDDE
:102AF000002010BDB461FF1F70B5040000F084FF1A
:102B000000230C200B4A010059438D18515C002909
:102B10000DD0A14208D1012300246B7000F014FEF7
:102B200000F05AFE200070BD01330A2BEBD11224B5
:102B3000F6E7C046B461FF1F70B5040000F064FF03
:102B4000002319001D000D4A1078002806D0A0426D
:102B50000CD1557001310C320A29F5D1002B0AD164
:102B600000F0A2FD00F038FE002070BD5078461E37
:102B7000B0411B18EEE700F0E7FDF3E7B461FF1F7B
:102B8000F7B504000C20002384460E4D01926746E1
:102B90005F43E85D7E19A04212D000280BD10A4B9A
:102BA0009C4662461B7808331370019B70707C55FD
:102BB0007160B360FEBD01330A2BE8D10320F9E751
:102BC0000720F7E7B461FF1FB061FF1F8020F8B551
:102BD000484BC0051B68C1248360474BFF251A681A
:102BE000012313434361454BA4001A68444B402121
:102BF0001A60444B1A68444B1A60444B1A59AA4352
:102C00001A51C52292009E58AE43314380269950F6
:102C10009F583F49F6010F403E439E509E588027E3
:102C20003602360A3043985080201A5900020A4072
:102C300002431A5104341A59364E3F04324080265A
:102C40003A431A511A5936061202120A32431A51DD
:102C500008341A5980260A4002431A51C3229200AE
:102C60009F58B446AF4337439F509F58294E0F405B
:102C700007439F509F5837408026360437438026AD
:102C80009F509F5836063F023F0A37439F50C0224D
:102C90001F59AF433A431A511A591202120A1643E6
:102CA000C6221E5192009C58AC4365462C439C5052
:102CB0009C5800250C4020439850C72080001A588B
:102CC000154C1140C02212020A431A50134B1B78B4
:102CD000DB08AB4201DC0020F8BD2378002B06D0D6
:102CE000A368002B00D0984701350C34EEE7122082
:102CF000F2E7C046D43DFF1FD03DFF1FB0F00040BB
:102D0000AC61FF1FB4F00040A861FF1F00E100E0CC
:102D1000FF00FFFFFFFF00FFB461FF1FB061FF1F57
:102D2000030010B51F2809D80722002013400724EC
:102D300004490A78A24313430B7010BD00230620F8
:102D4000F5E7C046B061FF1F054B06491B780A68CE
:102D500005485B0702401B0B134300200B607047C4
:102D6000B061FF1F1CF00040FFFFC1FF70B50C25D4
:102D7000FFF7EAFF0A4B1C780A4BE4086543ED189D
:102D8000002C01D1200070BD2B78002B06D06B6881
:102D9000002B00D09847013C0C3DF1E71220F2E7F0
:102DA000B061FF1FA861FF1F1FB5002102220B00A9
:102DB00001910091052000F0B7FD02230B490A683C
:102DC0001A42FCD120230393039B5A1E0392002B2B
:102DD000FAD1074A1368002BFCDA0B246C4420005C
:102DE000012100F001FD207804B010BD90C8004022
:102DF00000C8004013B504000A4B0193019B002B4F
:102E000001D1112016BDFFF7CFFF2300034004427C
:102E100005D0052000F078FD019B013BEDE718008F
:102E2000F0E7C046FFFFFF0707B500F0EDFD802289
:102E30000821D205936A0191002B01D107399162D3
:102E400002210C4A11600199481E01900029FAD113
:102E500003311160053101910199481E019000294B
:102E6000FAD11160002B02D18022D205936200F0CA
:102E7000B3FC07BD00C00040F0B52D4C89B02378ED
:102E8000002B4FD1FEF73EFD02232A4F03903A68F4
:102E90001A42FCD120230693069B5A1E0692002B51
:102EA000FAD1254E3368002BFCDA0120FFF7A2FF90
:102EB000011E02D0112009B0F0BD030003220190D1
:102EC000009005AD9F2000F02FFD0321280000F0A9
:102ED0008BFC02233A681A42FCD120230793079BFC
:102EE0005A1E0792002BFAD13368002BFCDA01201E
:102EF000FFF780FF0028DDD10398FEF717FDAA78C1
:102F00006B7811041B020B4329780B436360130099
:102F1000113B0A49052B07D801239340A3600B609E
:102F2000012323700020C6E780231B03F6E7C04679
:102F3000BC3DFF1F90C8004000C800409808FF1F1C
:102F40001E4B30B55A6818781D4B85B0D3185942BE
:102F50004B4101210093002300F036FD194B1A4A22
:102F600002259A6300221A6510325A658022C42114
:102F70009D65164B1648D202DA6789004258154BF8
:102F800080241A4080231B041343435064234120B0
:102F90000393E40500F006FA402000F003FA6562AE
:102FA000039D6B1E0393002DFAD103236362FFF789
:102FB0003BFFA562FFF760FF05B030BDC83DFF1FB6
:102FC00095FFFEF700C80040050001FF04E100E0A6
:102FD00000E100E0FFFF00FFF0B585B00700FEF75D
:102FE00091FC022305002D4C22681A42FCD12023BB
:102FF0000093009B5A1E0092002BFAD1284E336892
:10300000002BFCDA0120FFF7F5FE002803D0112485
:10301000200005B0F0BD234B2360022322681A4232
:10302000FCD120230193019B5A1E0192002BFAD15F
:103030003368002BFCDA0120FFF7DCFE0028E6D124
:10304000194B1F60022322681A42FCD120230293ED
:10305000029B5A1E0292002BFAD13368002BFCDA35
:103060000120FFF7C7FE0028D1D1104B23600223B7
:1030700022681A42FCD120230393039B5A1E039219
:10308000002BFAD13368002BFCDA0120FFF7B2FEE7
:10309000041EBCD12800FEF749FCB9E790C80040E7
:1030A00000C8004001000006A8C8004001800001DF
:1030B00010B50020FFF790FF10BD000010B5064BC3
:1030C00018705960FFF73CFF00211320034AFFF7F7
:1030D00057FD002010BDC046C83DFF1F412FFF1FF8
:1030E000F0B5040085B003920291FEF70BFC882234
:1030F00063035B0B52051A438023DB059D6A802323
:10310000274F0092BA68002601901B039A420CD9FF
:10311000F82326001B041E401C4206D08022214BAF
:1031200052025E6219680A431A60002D0BD100F04A
:103130006BFC02221C4B1A608023DB055A62013AA9
:103140009A6200F049FB0023039A934220D1002D9C
:103150000AD100F059FC144B03221D608023DB05CB
:103160005A629D6200F038FB8023BA681B039A42C2
:1031700008D9002E06D000220A4B0C495A621A6860
:103180000A401A600198FEF7D1FB002005B0F0BD9F
:10319000009A0299D2181278CA540133D4E7C04673
:1031A000BC3DFF1F00C8004000C00040FFFFFEFF05
:1031B000F0B587B0029103920400FEF7A3FB0190E3
:1031C00000F022FC802302250122234EDB0535601E
:1031D0005D629A6200F000FB204F3B682B42FCD1FD
:1031E00020230493049B5A1E0492002BFAD11C4DF9
:1031F0002B68002BFCDA0120FFF7FCFD002802D031
:10320000112007B0F0BD2000039A029900F02CFCB9
:10321000022304003A681A42FCD120230593059B3F
:103220005A1E0592002BFAD12B68002BFCDA0120E4
:10323000FFF7E0FD051EE3D100F0E6FB802303224B
:10324000DB0535605A629D6200F0C6FA0198FEF710
:103250006DFBE0B2D5E7C04600C0004090C800401A
:1032600000C80040F0B5802489B00600FEF74AFB94
:10327000E405A36A02250393029000F0C5FB012335
:10328000304F3D606562A36200F0A6FA2E4C2368C1
:103290002B42FCD120230593059B5A1E0592002B3F
:1032A000FAD12A4D2B68002BFCDA0120FFF7A2FD92
:1032B000002803D01124200009B0F0BD244B236066
:1032C000022322681A42FCD120230693069B5A1E31
:1032D0000692002BFAD12B68002BFCDA0120FFF7B5
:1032E00089FD021EE6D11B4B03211E6003000190E5
:1032F0000090202000F018FB022322681A42FCD123
:1033000020230793079B5A1E0792002BFAD12B68A4
:10331000002BFCDA0320FFF76DFD041ECAD100F07C
:1033200073FB80230322DB053C605A629C6200F041
:1033300053FA039B002B01D1FFF776FD0298FEF7AD
:10334000F5FAB8E700C0004090C8004000C800404F
:103350000100000694C8004007B500020191042254
:10336000000A01A9FFF724FF0EBD000073B5050098
:1033700005240B4AA3005B429B1819686B46DE1DAF
:103380003000FFF7B3FA022804D133782B55013C03
:10339000EFD276BD052CFCD00128FAD10230F8E737
:1033A000140900111F2807D8012380228340D20569
:1033B00091680B43936070473F2808D8012380220F
:1033C00020388340D20551690B435361F3E75F28EE
:1033D000F1D80123802240388340D205116A0B4383
:1033E0001362E8E71F2807D8012280218240C9051F
:1033F0008B6893438B6070473F2808D80122802157
:1034000020388240C9054B6993434B61F3E75F283D
:10341000F1D80122802140388240C9050B6A9343CC
:103420000B62E8E71F2810D880230200DB05153A5D
:103430001968012A06D820229143196019680A43A5
:103440001A60704701228240F6E73F2811D8802396
:103450000200DB05353AD968032A06D810229143C9
:10346000D960D9680A43DA60EBE70122203882404C
:10347000F5E75F28E5D842238022181A413B8340B4
:10348000D205516A99435162516A0B435362D8E79E
:1034900010B50400012813D1A022184992050B6829
:1034A0005B015B0913430B60154B164A1968114009
:1034B000154A0A431A60402219680A431A6010BD6F
:1034C0000028FCD101000A2000F09EF921000B2009
:1034D00000F09AF9C0220A4B920019680A43402171
:1034E0001A601A688A431A60B022044912060B68EF
:1034F0005B015B0913430B60E1E7C04614F0004039
:103500001CF000407F00FEFF80FD010072B6074AFC
:103510001368013313600422054B1A600023054A27
:1035200013608022D2055360FEE7C0467808FF1F73
:10353000C0F00040C4F0004005490B68002B05D1E5
:10354000044A0A6004490A60044A13607047C0468E
:10355000140AFF1F841E0000380AFF1FC4F0004039
:103560000023034A1360034A1360034A1360704741
:1035700054F0004040F1004044F10040002310B5F9
:10358000184C8AB0009301932378012B27D0694609
:10359000012000F029FA002817D1009B124902935C
:1035A000019B06AA0393114B02A81B680493104BBE
:1035B0001B68059300F068F910220E4906A800F078
:1035C0007BFA002804D1FF23237000200AB010BD2D
:1035D0000123094A074902A8237000F055F9012088
:1035E000F4E7C046B05EFF1F102900110829001142
:1035F0000C29001120290011B45EFF1F13B501240E
:103600006946012000F0F0F9034B00940193FFF7A5
:10361000B5FF200016BDC046BB0B000010B5FFF77C
:103620009FFFFFF7EBFF002802D0024B984710BD29
:10363000FEE7C046E1A2000002B471464908490015
:10364000095649008E4402BC7047C04602B4714618
:1036500049084900095C49008E4402BC7047C046D5
:1036600003B47146490840004900095A49008E4494
:1036700003BC70470000000001B40248844601BC4E
:10368000604700BFC1F7000001B40248844601BC96
:10369000604700BF49B5001101B40248844601BC2F
:1036A000604700BFE512010001B40248844601BC36
:1036B000604700BFADAE000001B40248844601BCC3
:1036C000604700BFBD0B010001B40248844601BC45
:1036D000604700BF090E000001B40248844601BCE7
:1036E000604700BF0934010001B40248844601BCB0
:1036F000604700BF8914010001B40248844601BC40
:10370000604700BF090E000001B40248844601BCB6
:10371000604700BFDD0A010001B40248844601BCD5
:10372000604700BFF535010001B40248844601BC82
:10373000604700BFD1AE000001B40248844601BC1E
:10374000604700BFF935010001B40248844601BC5E
:10375000604700BF21A9000001B40248844601BCB3
:10376000604700BF6911010001B40248844601BCF2
:10377000604700BF8552010001B40248844601BC85
:10378000604700BF8944000001B40248844601BC80
:10379000604700BFC95C010001B40248844601BC17
:1037A000604700BF8D11010001B40248844601BC8E
:1037B000604700BFE94C010001B40248844601BCE7
:1037C000604700BF0167010001B40248844601BCA4
:1037D000604700BF4DF9000001B40248844601BCB7
:1037E000604700BF9DA9000001B40248844601BCA7
:1037F000604700BF3D71010001B40248844601BC2E
:10380000604700BFB70E000001B40248844601BC07
:10381000604700BFF1A1001101B40248844601BC19
:10382000604700BFF90D010001B40248844601BCA5
:10383000604700BF71B0000001B40248844601BC7B
:10384000604700BF8512010001B40248844601BCF4
:10385000604700BFEDA5000001B40248844601BCEA
:10386000604700BFED68010001B40248844601BC16
:10387000604700BF016C010001B40248844601BCEE
:10388000604700BF01D7000001B40248844601BC74
:10389000604700BFDD3F000001B40248844601BC20
:1038A000604700BF6D0B010001B40248844601BCB3
:1038B000604700BFED6B010001B40248844601BCC3
:1038C000604700BF6137010001B40248844601BC73
:1038D000604700BFC115010001B40248844601BC25
:1038E000604700BF0134010001B40248844601BCB6
:1038F000604700BF6DF6000001B40248844601BC79
:10390000604700BFBD5C010001B40248844601BCB1
:10391000604700BF0189000001B40248844601BC31
:10392000604700BFE917010001B40248844601BCAA
:10393000604700BF496D010001B40248844601BCE4
:10394000604700BFD9B0000001B40248844601BC02
:10395000604700BFCD0C010001B40248844601BCA1
:10396000604700BF116E000001B40248844601BCEC
:10397000604700BF85C1000001B40248844601BC15
:10398000604700BFE90B010001B40248844601BC56
:10399000604700BFC166010001B40248844601BC13
:1039A000604700BFE927000001B40248844601BC1B
:1039B000604700BFD544010001B40248844601BC01
:1039C000604700BF2144000001B40248844601BCA6
:1039D000604700BFC56D010001B40248844601BCC8
:1039E000604700BF8D82000001B40248844601BCDC
:1039F000604700BFE1AC000001B40248844601BC4E
:103A0000604700BF7997000001B40248844601BCBA
:103A1000604700BF75A9000001B40248844601BC9C
:103A2000604700BF53B9000001B40248844601BC9E
:103A3000604700BF7912010001B40248844601BC0E
:103A4000604700BF5976010001B40248844601BCBA
:103A5000604700BF51B8000001B40248844601BC71
:103A6000604700BF156B010001B40248844601BCE9
:103A7000604700BF9573010001B40248844601BC51
:103A8000604700BFDD0C010001B40248844601BC60
:103A9000604700BFC9A9000001B40248844601BCC8
:103AA000604700BFE9D4000001B40248844601BC6D
:103AB000604700BF2D6C010001B40248844601BC80
:103AC000604700BFCD4C010001B40248844601BCF0
:083AD000604700BF053401004E
:103AD80002000000DEBD001101000000F0BB001173
:103AE80002000000DABD001101000000183BFF1FB2
:103AF80002000000F8BB001101000000285CFF1F55
:103B080002000000D8BD0011030000009C5BFF1FED
:103B18001200000002000000DEBD001101000000DC
:103B280038BC001102000000DABD001101000000DD
:103B380035BC00110200000042BC00110300000067
:103B4800D75BFF1F02000000D8BD00110300000072
:103B5800EC5BFF1F02000000DABD0011010000004D
:103B680034BC00110200000040BC0011030000003A
:103B7800AD5BFF1F02000000D8BD0011030000006C
:103B8800CE5BFF1F02000000DEBD00110100000037
:103B980078BC001102000000DABD0011010000002D
:103BA800613CFF1F020000008ABC001101000000F8
:103BB80073BC001102000000DABD00110100000012
:103BC800603CFF1F0200000088BC001101000000DB
:103BD800F45BFF1F02000000DABD001101000000C5
:103BE8005F3CFF1F0200000086BC001101000000BE
:103BF80063BC001102000000DABD001101000000E2
:103C08005E3CFF1F0200000084BC001101000000A0
:103C18005EBC001102000000DABD001101000000C6
:103C28005D3CFF1F0200000082BC00110100000083
:103C380059BC001102000000DABD001101000000AB
:103C48005C3CFF1F0200000080BC00110100000066
:103C580054BC00110202020202020000000000002F
:103C68000D0C0000994B00115F4B0011CCBC0011EA
:103C780090011D0018001800FFFF0701020304054A
:103C8800060201060000000000000000000000001D
:103C9800000000000000000000000000000000001C
:103CA8000300000002000000DEBD0011010000005A
:103CB800ECBC001102000000DABD00110100000098
:103CC8001C3DFF1F02000000F6BC001101000000AF
:103CD800225CFF1F02000000D8BD00110300000095
:103CE8008C5EFF1F02000000DABD00110100000019
:103CF8001C3DFF1F02000000F4BC00110100000081
:103D0800245CFF1F02000000D8BD00110300000062
:103D1800845EFF1F126C6C6C0000000000580040AD
:103D2800151600000001000000000111FFFF00004F
:103D38005048593600000000000000000B00050044
:103D4800F0000000B4000028002800283075A0000A
:103D5800A000A000A00000080008E001F00010008A
:103D6800100010001000100010005000500050000B
:103D780010001000D0070000000000000F00010034
:103D88000500307507001000010081FF00000000E9
:103D9800FF000000D9730011E1710011716F00116B
:103DA800FFFF0100FF000000F59D0011719B00114D
:103DB800899A0011000000000000000000000800BF
:103DC800040000003B0001085902E0018821280096
:103DD80002000000DEBD001101000000A4BE0011B9
:103DE80002000000DABD001101000000553EFF1F6F
:103DF80002000000D6BD0011010000006C62FF1F28
:103E080002000000DABD001101000000543EFF1F4F
:103E180002000000D4BD001101000000523EFF1F47
:103E280002000000DABD001101000000503EFF1F33
:103E380002000000D2BD001101000000483EFF1F33
:103E4800180018001D009001020000030202000083
:103E580002000000DEBD001101000000B8BE001124
:103E680002000000DABD001101000000983EFF1FAB
:103E780002000000D0BD001100000000000000009A
:103E880002000000D8BD0011030000008C62FF1F73
:023E980020FF09
:040000051FFF184180
:00000001FF
